:020000040000FA
:10000000503D002001850000258500002785000067
:10001000298500002B8500002D8500002F8500001C
:100020002F8500002F8500002F8500002F85000000
:100030002F8500002F8500001F800000D382000064
:10004000034800000D480000174800002148000048
:100050002B480000354800003F4800004948000098
:10006000534800005D4800006748000071480000E8
:100070007B480000854800008F4800009948000038
:10008000A3480000AD480000B7480000C148000088
:10009000CB480000D5480000DF480000E9480000D8
:1000A000F3480000FD480000074900001149000026
:1000B0001B490000254900002F4900003949000074
:1000C000434900004D4900005749000061490000C4
:1000D0006B490000754900007F4900008949000014
:1000E000934900009D490000A7490000B149000064
:1000F000BB490000C5490000CF490000D9490000B4
:10010000E3490000ED490000F7490000014A000002
:100110000B4A0000154A00001F4A0000294A00004F
:10012000334A00003D4A0000474A0000514A00009F
:100130005B4A0000654A00006F4A0000794A0000EF
:10014000834A00008D4A0000974A0000A14A00003F
:10015000AB4A0000B54A0000BF4A0000C94A00008F
:10016000D34A0000DD4A0000E74A0000F14A0000DF
:10017000FB4A0000054B00000F4B0000194B00002C
:10018000234B00002D4B0000374B0000414B00007B
:100190004B4B0000554B00005F4B0000694B0000CB
:1001A000734B0000854B00008F4B0000994B000003
:1001B000A34B0000AD4B0000B74B0000C14B00004B
:1001C000CB4B0000D54B0000DF4B0000E94B00009B
:1001D000F34B0000FD4B0000074C0000114C0000E9
:1001E0001B4C0000254C00002F4C0000394C000037
:1001F000434C00004D4C0000574C0000614C000087
:10020000DFF80CD009F056FF00480047F39E0000CD
:10021000503D0020EFF3108072B67047EFF310806E
:100220007047EFF3108062B6704730BF704780F3BD
:1002300011887047EFF31180704700000138FDD13D
:100240007047000030B50246F74B1824F7480068A5
:10025000F74D2840F74DA84201D1F74B1B24002150
:1002600008E053F83100904203D103EBC10040682D
:1002700030BD491CA142F4D30020F9E702F001038C
:100280001BB1D0F800340B4302E0D0F800348B43AC
:10029000C0F8003402F002031BB1D0F820340B4345
:1002A00002E0D0F820348B43C0F82034704730B5DA
:1002B000024601208840C1B2D2F80034D2F820446E
:1002C00003EA010008B1012000E0002004EA010572
:1002D0000DB1022500E00025284330BD02F00103E6
:1002E0001BB1D0F808340B4302E0D0F808348B433C
:1002F000C0F8083402F002031BB1D0F804340B43F9
:1003000002E0D0F804348B43C0F8043402F0040354
:100310001BB1D0F80C340B4302E0D0F80C348B4303
:10032000C0F80C3402F4803323B1D0F8383543F0F0
:10033000010303E0D0F8383523F00103C0F8383565
:100340007047F0B5024601208840C1B2D2F80834A7
:10035000D2F80444D2F80C64D2F8385503EA01000C
:1003600008B1012000E0002004EA01070FB10227D4
:1003700000E00027384306EA01070FB1042700E038
:100380000027384305F0010717B14FF4803700E02C
:1003900000273843F0BDF0B5A44D2D68A44E35407C
:1003A000A64EB5421AD0002416E00125A5400D4006
:1003B00085B1D0F8C45F67000326BE40B543C0F8DE
:1003C000C45FD0F8C45F6700C2F34116BE40354336
:1003D000C0F8C45F651CECB2082CE6DB02F0010536
:1003E0001DB1D0F800550D4302E0D0F800558D4303
:1003F000C0F8005502F002051DB1D0F804550D43B8
:1004000002E0D0F804558D43C0F8045502F004050D
:100410001DB1D0F808550D4302E0D0F808558D43C2
:10042000C0F8085502F008051DB1D0F818550D4365
:1004300002E0D0F818558D43C0F818557B4D2D6853
:100440007B4E35407D4EB5420BD002F010051DB1FC
:10045000D0F83C550D4302E0D0F83C558D43C0F830
:100460003C5503F001051DB1D0F80C550D4302E0D9
:10047000D0F80C558D43C0F80C5503F002051DB1A2
:10048000D0F810550D4302E0D0F810558D43C0F858
:10049000105503F004051DB1D0F814550D4302E0CA
:1004A000D0F814558D43C0F8145503F008051DB15C
:1004B000D0F81C550D4302E0D0F81C558D43C0F810
:1004C0001C555A4D2D685A4E35405C4EB54217D0DA
:1004D00003F400751DB1D0F844550D4302E0D0F887
:1004E00044558D43C0F8445503F440751DB1D0F810
:1004F00040550D4302E0D0F840558D43C0F84055BB
:100500001BB9D0F828550D4302E0D0F828558D438B
:10051000C0F82855F0BDF0B514461D4601268E40A2
:10052000F1B2D0F800650E400EB1012600E00026C1
:100530003246D0F804650E400EB1022600E00026D7
:100540003243D0F808650E400EB1042600E00026C4
:100550003243D0F818650E400EB1082600E00026A0
:100560003243324E3668324F3E40344FBE420FD097
:10057000D0F83C650E400EB1102600E00026324354
:10058000D0F8C46F4F00FE4006F0030642EA461260
:100590002260D0F80C650E400EB1012600E0002666
:1005A0003346D0F810650E400EB1022600E000265A
:1005B0003343D0F814650E400EB1042600E0002647
:1005C0003343D0F81C650E400EB1082600E000262B
:1005D0003343164E3668164F3E40184FBE420CD07D
:1005E000D0F840650E4046B1D0F844650E400EB1DB
:1005F000FE1401E04FF4807633432B60F0BDD0F859
:1006000010240A43C0F810247047D0F810248A43FD
:10061000C0F810247047024611B1D2F81804704790
:10062000D2F81404FBE70000A8A4000000E00F408B
:100630000000FF7000000A1068A50000000005100F
:10064000C0F81C14704770B504460D462046FFF7ED
:10065000F9FD06462946304600F006FC304600F01B
:100660005FFC70BD70B504462046FFF7EBFD054604
:10067000284600F091FC284600F010FC70BD2DE9E2
:10068000F04107460C4615463846FFF7DBFD0646A7
:100690003019294600F0E8FB301900F041FCBDE8B4
:1006A000F08170B506460C463046FFF7CBFD054697
:1006B000281900F071FC281900F0F0FB70BD02460B
:1006C000002000EB810010587047002303EB8103EA
:1006D000C250704730B504460D46002229462046D8
:1006E000FFF7CCFD0023012229462046FFF753FEE9
:1006F00030BD30B504460D46022229462046FFF79C
:10070000BDFD0823662229462046FFF744FE30BD82
:1007100030B504460D46002229462046FFF7AEFDBF
:100720000023012229462046FFF735FE30BD30B5B3
:1007300004460D46022229462046FFF79FFD082366
:10074000012229462046FFF726FE30BD30B504467B
:100750000D46022229462046FFF790FD082301227C
:1007600029462046FFF717FE30BD30B504460D463A
:10077000022229462046FFF781FD082366222946EA
:100780002046FFF708FE30BD30B504460D46022274
:1007900029462046FFF772FD082366222946204697
:1007A000FFF7F9FD30BD30B504460D46022229465B
:1007B0002046FFF763FD0823662229462046FFF7FF
:1007C000EAFD30BD30B504460D46002229462046DC
:1007D000FFF754FD0823012229462046FFF7DBFDE1
:1007E00030BD30B504460D46082301222946204677
:1007F000FFF7D1FD012229462046FFF73FFD30BD1E
:1008000030B504460D460923012229462046FFF74C
:10081000C2FD012229462046FFF730FD30BD30B52C
:1008200004460D46022229462046FFF727FD0823ED
:10083000012229462046FFF7AEFD30BD30B5044603
:100840000D46022229462046FFF718FD0923012202
:1008500029462046FFF79FFD30BD30B504460D46C2
:10086000022229462046FFF709FD082301222946D6
:100870002046FFF790FD30BD30B504460D460222FC
:1008800029462046FFF7FAFC08236622294620461F
:10089000FFF781FD30BD30B504460D4602222946E2
:1008A0002046FFF7EBFC0823012229462046FFF7EC
:1008B00072FD30BD30B504460D4602222946204661
:1008C000FFF7DCFC0823012229462046FFF763FDE1
:1008D00030BD30B504460D46022229462046FFF7BA
:1008E000CDFC0A23012229462046FFF754FD30BDE6
:1008F00030B504460D46022229462046FFF7BEFCCD
:100900000823012229462046FFF745FD30BD30B5BA
:1009100004460D46022229462046FFF7AFFC082375
:10092000012229462046FFF736FD30BD30B504468A
:100930000D46022229462046FFF7A0FC082301228B
:1009400029462046FFF727FD30BD30B504460D4649
:10095000022229462046FFF791FC0823012229465E
:100960002046FFF718FD30BD30B504460D46002285
:1009700029462046FFF782FC002301222946204613
:10098000FFF709FD30BD30B504460D460222294669
:100990002046FFF773FC0823012229462046FFF773
:1009A000FAFC30BD30B504460D46002229462046EB
:1009B000FFF764FC4FF40273012229462046FFF73B
:1009C000EAFC30BD30B504460D46002229462046DB
:1009D000FFF754FC4FF48473012229462046FFF7A9
:1009E000DAFC30BD0146D1F84805704710B5014624
:1009F000C1F307401F4BDB6E01248440234033B119
:100A0000012303EB40031C4C54F8230003E0430094
:100A1000194C54F82300C1F30722D0F82C350F24C9
:100A20009440A34301F00F0494402343C0F82C35B5
:100A300010BDD0F834250A43C0F834257047D0F8EB
:100A400034258A43C0F834257047D0F830250A434E
:100A5000C0F830257047D0F830258A43C0F83025DB
:100A60007047064AC0F82025D0F824250A43C0F86C
:100A70002425704700E00F4040A600004B434F4C38
:100A800030B50246E64B0624E6480068E64D2840AD
:100A9000E64DA84201D1E64B0A24002108E053F8B4
:100AA0003100904203D103EBC100406830BD491CC6
:100AB000A142F4DB0020F9E7016A41F01001016274
:100AC000704770B503460C4616461846FFF7F4FF0C
:100AD000012E01D1D74A00E0D74A142000FB024082
:100AE000401E02EB82018900B0FBF1F0451EDD6083
:100AF000D3F8C00F00F0010048B1D0482044401E98
:100B0000CE49B0FBF1F0451E45F08000D86070BDC5
:100B1000016A41F0200101620121C0F80418704708
:100B200000B502460B461046FFF7F2FFC2F8003848
:100B300000BD11B1012908D102E0C0F8002804E08D
:100B400042F08003C0F81C3800BF00BF7047016A44
:100B500021F01001016270470021C0F80418016AF9
:100B600021F020010162704770B504460D46204611
:100B7000FFF786FF06462946304600F075F93046F5
:100B800000F0CEF970BD70B504462046FFF778FF3F
:100B90000546284600F000FA284600F07FF970BDAF
:100BA00001210161704702690A4302617047D0F870
:100BB0000C1841F00101C0F80C187047D0F80C284F
:100BC0000A43C0F80C287047002101617047026990
:100BD0008A4302617047D0F80C1821F00101C0F877
:100BE0000C187047D0F80C288A43C0F80C287047BE
:100BF000024629B1906908B1012070470020FCE746
:100C0000506908B10120F8E70020F6E7024609B173
:100C1000906970475069FCE7024631B1D2F8140878
:100C200008B1012070470020FCE7D2F8100808B195
:100C30000120F7E70020F5E7024611B1D2F81408C9
:100C40007047D2F81008FBE70121C161816170474C
:100C5000C16170470121C0F818187047C0F8181812
:100C6000704742EA4103036070470146C86A704713
:100C70000146486800F0010008B1012070470020DB
:100C8000FCE70146486800F0400008B101207047C9
:100C90000020FCE7416070470246516801F0010006
:100CA00008B10020704701F0120010B101F01C00E3
:100CB000F8E70020F6E781607047014688687047D2
:100CC0004162704731B1D0F8202842F00102C0F8EB
:100CD000202805E0D0F8202822F00102C0F82028C2
:100CE000704731B1D0F8202822F00202C0F8202845
:100CF00005E0D0F8202842F00202C0F82028704712
:100D00000146D1F804087047C0F80818704701463A
:100D1000D1F808087047D0F8042F6FF30F02C0F81D
:100D2000042FD0F8042F0A43C0F8042F7047D0F8DE
:100D3000041F41F48041C0F8041F7047D0F8042F0D
:100D400092B2C0F8042FD0F8042F0A43C0F8042F41
:100D50007047D0F8041F41F08041C0F8041F70476D
:100D60000146D1F8080F704700BFD0F8082F02F0F5
:100D70000202002AF9D1C0F8001F70470246D2F8DB
:100D8000080F00F0020008B100207047C2F8001FF1
:100D90000120FAE7014600BFD1F8080F00F48030C7
:100DA0000028F9D1D1F8000F70470246D2F8080F99
:100DB00000F4803008B100207047D2F8000F0870AE
:100DC0000120F9E7016370470146486B7047154AF7
:100DD0001268154B1A40154B9A4202D1C2680A4359
:100DE000C260104A1268104B1A40154B9A4207D144
:100DF000826B42EA11328263026A42F0400202626E
:100E0000704741F00102C0F8042870470121C0F882
:100E100004187047016A41F0010101627047000047
:100E2000D0A6000000E00F400000FF7000000A1094
:100E300000A70000801A0600A08601008047370145
:100E40000000051000BFFEE710B5FFF7EAF908B192
:100E5000012010BD0020FCE710B5FFF7DBF908B159
:100E6000012010BD0020FCE730B50246B64C2468D6
:100E7000B64DAC420ED0B44C2368002005E053F8C8
:100E80002040B24D45F82040401C9B28F7D3AF4C82
:100E9000AD4D2C60AD4C44F8221030BDAC49AB4A8E
:100EA00042F820107047AB4951F82010AA4A11436C
:100EB000A54A121D11607047A34A121D126802F460
:100EC000E061002006E0A34A52F820208A4200D1C7
:100ED00002E0401C0828F6D300BF704710B50A4650
:100EE00083089E4C54F8233019688307DC0EFF23D7
:100EF000A34099438307DB0E02FA03F319438308E7
:100F0000964C54F82330196010BD01468808934A66
:100F100052F8200000688A07D20ED040C0B2704755
:100F2000042808D188491C31096841F48031864A77
:100F30001C3211602FE0052808D183491C31096853
:100F400041F40031804A1C32116024E0062808D1A7
:100F50007D491C31096841F480217B4A1C321160B3
:100F600019E00F2808D14FF0E021096941F0020192
:100F70004FF0E02211610EE010280CD3A0F1100117
:100F800001F01F0201219140A0F110025209744B9F
:100F900053F8222011607047042808D16A491C3197
:100FA000096821F48031684A1C3211602FE005285D
:100FB00008D165491C31096821F40031624A1C32AC
:100FC000116024E0062808D15F491C31096821F42A
:100FD00080215D4A1C32116019E00F2808D14FF0C2
:100FE000E021096921F002014FF0E02211610EE0D9
:100FF00010280CD3A0F1100101F01F020121914033
:10100000A0F110025209574B53F82220116070478B
:1010100010B501460020042905D14B4A1C32126844
:1010200002F4803028E0052905D1474A1C321268B5
:1010300002F4003020E0062905D1434A1C32126830
:1010400002F4802018E00F2905D14FF0E022126948
:1010500002F0020010E010290ED3A1F11002520993
:101060003F4B53F822201268A1F1100303F01F0434
:101070000123A34002EA030010BD022808D132492F
:10108000091F096841F000412F4A121F116024E036
:101090000E2808D12C49091F096841F080512A4ABD
:1010A000121F116019E00F2808D12749091F09688C
:1010B00041F08061244A121F11600EE010280CD309
:1010C000A0F1100101F01F0201219140A0F11002D6
:1010D0005209254B53F82220116070470E2808D181
:1010E0001949091F096841F00061174A121F116070
:1010F00019E00F2808D11449091F096841F000714F
:10110000114A121F11600EE010280CD3A0F110013B
:1011100001F01F0201219140A0F110025209134B6E
:1011200053F822201160704710B504462046FFF79F
:101130007EF810BD10B5FFF77DF810BDA0F11001CD
:101140000B4A11607047000008ED00E00004002029
:10115000450E000050A700000000FA0570A700002F
:101160000CA8000020A8000034A8000048A8000037
:1011700000EF00E0024600210AE0F74850F8310095
:10118000904204D3F44800EBC10040687047491C0A
:101190000629F2D30020F9E7F0B50146DFF8BCC319
:1011A000DCF860C1CCF38923DFF8B0C3DCF860C1A0
:1011B000CCF30905DFF8A4C3DCF864C1CCF3042C3C
:1011C0000CF10106DFF894C3DCF864C10CF01F0CCD
:1011D0000CF10107B1FBF7F15A09A3EB421401FB33
:1011E00005F001FB02FC00EB5C1001FB04FC00EBD2
:1011F0009C20B0FBF6F0F0BDD8483C380068401C9D
:1012000000027047D5480068D5490840D549884252
:1012100006D1D24880680004400900F5006070479C
:10122000CE484038006880B2401CC002F7E7CB4887
:101230000068CB490840CC49884209D1C7484038AA
:101240000068C0F302400A30012101FA00F0704743
:101250004FF48060FBE70146C1F30720C34A104406
:1012600000F0704040F00070C1F30722BF4B1A44F9
:10127000C2F3130240EA4210CAB240EA8200006898
:1012800008B1012070470020FCE70146C1F30720A8
:10129000B74A104400F0704040F00070C1F30722DC
:1012A000B34B1A44C2F3130240EA4210CAB240EAF6
:1012B0008200006808B1012070470020FCE710B5EB
:1012C0000121C0F30722AB4B1A4402F0704242F0F6
:1012D0000072C0F30723A74C2344C3F3130342EA6D
:1012E0004312C3B242EA8302116010BD10B500215F
:1012F000C0F307229F4B1A4402F0704242F0007282
:10130000C0F307239B4C2344C3F3130342EA431265
:10131000C3B242EA8302116010BD18B50121C0F3C7
:101320000722954B1A4402F0704242F00072C0F35B
:101330000723914C2344C3F3130342EA4312C3B27D
:1013400042EA830211600021009102E00099491CE9
:10135000009100991029F9D30021C0F30722864B90
:101360001A4402F0704242F00072C0F30723824C2C
:101370002344C3F3130342EA4312C3B242EA830293
:10138000116018BD10B50121C0F307227B4B1A4430
:1013900002F0704242F00072C0F30723774C2344FE
:1013A000C3F3130342EA4312C3B242EA8302116059
:1013B00010BD10B50021C0F30722704B1A4402F093
:1013C000704242F00072C0F307236C4C2344C3F315
:1013D000130342EA4312C3B242EA8302116010BD12
:1013E00010B50121C0F30722654B1A4402F0704288
:1013F00042F00072C0F30723614C2344C3F313038C
:1014000042EA4312C3B242EA8302116010BD10B532
:101410000021C0F307225A4B1A4402F0704242F0F6
:101420000072C0F30723564C2344C3F3130342EA6C
:101430004312C3B242EA8302116010BD10B501210C
:10144000C0F307224F4B1A4402F0704242F0007280
:10145000C0F307234B4C2344C3F3130342EA431264
:10146000C3B242EA8302116010BD10B50021C0F37F
:101470000722444B1A4402F0704242F00072C0F35B
:101480000723404C2344C3F3130342EA4312C3B27D
:1014900042EA8302116010BD30490968304A1140A8
:1014A000304A91420ED130B12C49096E41F00061B1
:1014B0002A4A116618E02949096E21F00061274A7D
:1014C000116611E040B12549B031096841F0005181
:1014D000224AC2F8B01007E02049B031096821F073
:1014E00000511E4AC2F8B010704710B5044621469C
:1014F0002C20FFF7B9FC2C20FFF712FD10BD10B512
:101500002C20FFF749FD2C20FFF7C8FC10BD134924
:10151000496D0143114A516570471049496D814336
:101520000E4A516570470D4988657047014611B1F3
:101530000A48806D70470948006DFBE71249086052
:1015400070471148006870470F49083108607047BC
:101550000D4808300068704778AA000000E00F408E
:101560000000FF700000051000000A1000E30F40AB
:1015700000EA0F4000E90F4000E50F4000E60F4091
:1015800000E70F4000E80F40B4E10F40FE4908605B
:101590007047FD49091D08607047FC48FC49086018
:1015A00000BFFEE710B5FEF740FE10BD10B5F848CD
:1015B000001D006840F00400F549091D0860FEF7B1
:1015C00034FEF348001D006820F00400F049091DB6
:1015D000086010BDEF48C06D7047EE49C96D81438A
:1015E000EC4AD1657047EB49C86770470146EA4845
:1015F000084050B101F00040E34A383A1060E64834
:1016000081380840E34AC2F85001DF4838380160A9
:1016100001F4007088B100BFDB483438006800F482
:1016200040700028F8D0D8483438006800F4407082
:10163000B0F5807F01D0002070470120FCE7D2493F
:10164000503108607047D0485030006870472DE92D
:10165000FE4F05468A46CF480068D0490840D04929
:10166000884202D10020BDE8FE8FC5F3841705F043
:101670003800102805D1DFF82C93002600BF15276D
:1016800048E005F03800302804D147F230594FF4D3
:1016900000163FE005F03800382804D14FF4004927
:1016A0004FF4800636E005F0380078BB1A2F01DCD5
:1016B000092F01DA0020D6E7BB4850F827904FF4F5
:1016C000401646F04076B348C06F20F01C000190F1
:1016D000072F03DB019840F010000190AD490198FD
:1016E000C8674FF40020009005E00098401E00906D
:1016F000009800B905E0A748006D00F4807000284C
:10170000F3D000BF009828B90020ACE7FFE74FF006
:101710000009002605F46050002874D105F0380057
:1017200028B105F03800102801D000209BE7C5F350
:10173000026002909D48FFF71DFD9649C031086088
:101740009448D0F8B0009A4900EA010444F00044FB
:101750009048B0300460093F9649029851F8200043
:101760005044401EB0FBFAF88A48D0F8B00030432D
:101770008849B0310860029800EBC00000EB4000DF
:101780008D4901EBC00007EB470100EB8100406889
:101790008049C1F864017C4824380168A8F101003F
:1017A00041EA00207B49C1F86401029800EBC000C7
:1017B00000EB4000804901EBC00007EB470150F807
:1017C000210071492839096801F4000108436E4974
:1017D000283908604846FFF7DFFC4FEA500A5046B8
:1017E000FFF7C8FC6B49C1F8C0000846D0F860019B
:1017F00000F4000040B16748B030006840F080401D
:10180000C1F8B00008E02BE05F482838006840F4D9
:1018100000006049C1F860014FF4004B08E05A48ED
:101820002038006800F0010000B104E0ABF1010BCA
:10183000BBF1000FF3DC00BFBBF1000F0DD055482A
:10184000B030046846F0010040F08050044344F09A
:1018500000445048C0F8B0403CE04FF0000A39E086
:101860005048FFF787FC4B49C03108604948D0F821
:10187000600120F400004749C1F860010846D0F833
:10188000B0404E48044044F000444248B030046048
:10189000BAF1000F02D14FF000080AE0B9FBFAF8E4
:1018A000B8F1000F01D0A8F1010808F10100B9FB5F
:1018B000F0FA5046FFF75EFC3649C0310860354803
:1018C000D0F8B04046EA8820044344F00044314850
:1018D000B03004602F48B030006820F470002D490B
:1018E000C1F8B0005046BEE62DE9F0410646294851
:1018F000046E056F44F4006424F4800445F400652C
:101900000466056704F00100D8B106F00100C0B913
:1019100066F0010004404FF480701E498865084657
:1019200004664FF4002702E07F1E07B905E019485E
:10193000006D00F480700028F6D000BF0FB9BDE83C
:10194000F08124F4FE6406F4FE6004431C48054064
:101950001B49A13106EA0100054306F0080045EAEB
:10196000C0050C480466056724F4005406F40050D2
:10197000044325F4005506F4005005434020054972
:10198000886505F000401DE088E10F400400FA057D
:101990000CED00E000E00F40000100800000FF704F
:1019A000000005100024F4005CA8000040787D01D0
:1019B00000FC0FE0A8AA0000C8A80000FF0300EF89
:1019C0008FFFFF7F18B108460567046602E0D6481E
:1019D00004660567D5480440C14306EA0100044394
:1019E00025F0FC5506F0FC50054306F0804040B160
:1019F00044F4800425F48005CD4906EA010005433E
:101A000001E025F0804506F4006080B94FF40047FE
:101A100006E0C848006800F0010000B102E07F1E47
:101A2000002FF6D100BF24F4006425F40065BE4801
:101A3000046605671020FEF701FC00BF7FE7F0B5E4
:101A4000B948036E026F02F0004010B102F070005E
:101A500001E003F03000202811D003DC38B1102859
:101A600015D10AE030280CD0702810D10CE0B24813
:101A7000C3F3841750F827100BE0B04909E0B049D0
:101A800007E047F2305104E04FF4004101E000204C
:101A9000F0BD00BF4FF0FF3402F0004010B102F47F
:101AA000006028B102F0004098BB03F4006080BBE6
:101AB000A048083805689C48D0F8646106F01F000B
:101AC000401CC6F304277F1C10FB07F04000B1FB4D
:101AD000F0F1C5F309004843C5F389274F4300EBF4
:101AE000972143F480039048006900F47040B0F5FA
:101AF000804F13D006DCB0F5005F0BD0B0F5405F2F
:101B000012D109E0B0F5E04F0AD0B0F5104F0BD17B
:101B100008E00BE08B4C08E08B4C06E08B4C04E0BB
:101B20008B4C02E08B4C00E000BF00BF03F4800050
:101B300018B302F00040D8B102F0804090B102F03A
:101B4000004010B102F4006028B102F0004048B932
:101B500003F4006030B94F00C2F38650401CB7FB5D
:101B6000F0F10AE0C2F3C550401CB1FBF0F104E013
:101B7000C3F3C350401CB1FBF0F18C4200D22146AC
:101B8000084685E76B4924390860704710B502465E
:101B9000654B1B68704C2340704CA34208D121F068
:101BA000FC54531E44EAC353624C243C236023E09C
:101BB000501E01F0700333B1102B0ED0302B05D026
:101BC000702B09D105E040F4401007E040F400100C
:101BD00004E040F4800001E000BF00BF00BF01F05E
:101BE00002030BB140F0004001F080430BB140F024
:101BF0008040504B243B186010BD4B49096E21F4C6
:101C0000F0110143484A116670474748006E00F4DE
:101C1000801008B9002070474348006E00F4F010AF
:101C2000F9E74149C96E00F00F0301229A401143C0
:101C30003D4AD16670473C49C96E00F00F0301224E
:101C40009A409143384AD16670473748006F20F474
:101C500080403549086770473348006F40F4804042
:101C60003149086770473049886370472E48006ED5
:101C700070472D49096E01432B4A116670472DE9C3
:101C8000F04F054628480068DFF8CCE000EA0E0077
:101C9000DFF8C8E0704503D100200860BDE8F08F90
:101CA0002148B030076807F08050B0F1805F02D063
:101CB00000200860F2E7C5F384161F4850F826405C
:101CC0001C48083802681848D0F86431C2F3090C7F
:101CD000C2F3892803F01F09C3F3042A04FB0CF0A4
:101CE00004FB08FE00EB9E2B09F101000AF1010E36
:101CF00010FB0EF0BBFBF0FBC1F800B00120CDE7FC
:101D00000948406E70470849496E8143064A51664A
:101D100070474A1ED2B20243064B203B1A607047FE
:101D2000044930390860704700E00F40FEFF3FF87B
:101D30000000404068E10F405CA800000024F4006F
:101D400000093D0000B4C40480F0FA02005A6202A7
:101D500040787D01002D31010000FF70000005106A
:101D600030B50246C74B0824C7480068C74D284015
:101D7000C74DA84201D1C74B00BF002108E053F86E
:101D80003100904203D103EBC100406830BD491CD3
:101D9000A142F4D30020F9E7C26A22F086020A4386
:101DA000C26270470146C86A00F08600704741EA87
:101DB00002034363704710B5436B03F007040C60E4
:101DC00003F03804146010BDC16A41F01001C16213
:101DD000016B40F2013211430163704700BF81691A
:101DE00001F008010029FAD1C16A21F01001C16295
:101DF000016B40F20132914301637047F0B5044634
:101E00000E4615461F462046FFF7E8FFB6EB051FB6
:101E100005D2206B40F0200020636D0803E0206BAA
:101E200020F020002063F000B0FBF5F0401C4308D8
:101E30009809606203F03F00A062E7620020A061A1
:101E40002046FFF7C1FFF0BDF0B5446A856A8E00F9
:101E5000402707FB0457B6FBF7F61660066B06F043
:101E6000200616B1166876001660C66A06F0EE0601
:101E70001E60F0BDC16A41F01001C1627047C16AC5
:101E800021F01001C162704721B1026B42F00602DD
:101E9000026303E0026B42F0020202637047016BCF
:101EA00021F0060101637047C16A21F0E60141F0AB
:101EB0006E01C162026B42F0080202637047016B5F
:101EC00021F0080101637047026B01F440631A437B
:101ED00002637047026B01F440639A4302637047E8
:101EE0000146086B00F4406070470146886940F283
:101EF000071210407047026B22F440420A4302630B
:101F000070470146086B00F440407047026B22F0B6
:101F100010020A43026370470146086B00F010008C
:101F2000704701468869012222EA10107047014675
:101F30008869012222EA501070470146886900F042
:101F4000100008B9086870474FF0FF30FBE7014602
:101F500000BF886900F010000028FAD108687047B7
:101F60000246906900F0200010B91160012070470E
:101F70000020FCE700BF826902F02002002AFAD1AB
:101F80000160704719B1C26A42F0010202E0C26A00
:101F900022F00102C262704701468869C0F3C000A6
:101FA000704770B504460D462046FFF7D9FE064639
:101FB00029463046FEF758FF3046FEF7B1FF70BDA8
:101FC00070B504462046FFF7CBFE05462846FEF7CF
:101FD000E3FF2846FEF762FF70BD826B0A4382630F
:101FE0007047826B8A4382637047024609B1106C66
:101FF0007047D06BFCE741647047826C0A4382648F
:102000007047826C8A43826470470146486800F0DA
:102010000F007047002141607047C0F8C81F70472B
:102020000146D1F8C80F7047D0F8A41041F4004120
:10203000C0F8A4107047D0F8A41021F40041C0F8F3
:10204000A4107047C0F8A410C0F8A82070470A4632
:1020500000BF836903F08803802BFAD1C16A21F0A5
:10206000040343F08203C362026000BF836903F08C
:102070008803802BFAD1C1627047016B41F0800167
:1020800001637047B0AA000000E00F400000FF703D
:1020900000000A10F0AA000072B6704762B67047DE
:1020A000EFF3108072B6704780F31088704730BF2E
:1020B000704720BF7047B0FA80F0704790FAA0F0E8
:1020C000B0FA80F0704790FAA0F0704710B5B0F108
:1020D000005F0AD3FE4CA04207D8440104EB810301
:1020E00003F10852002414600CE0B0F1804F09D3D2
:1020F000F84CA04206D8440104EB810303F184426A
:102100000024146010BD10B5B0F1005F0AD3F04C8C
:10211000A04207D8440104EB810303F108520124D3
:1021200014600CE0B0F1804F09D3EA4CA04206D80D
:10213000440104EB810303F184420124146010BDC7
:102140002DE9F04104464FF00008102C6BD2DFE877
:1021500004F0080E0F1014293E090A0B0C11120D81
:10216000135300BF00BF00BF00BF00BF89E000BF26
:1021700000BF00BF00BF00BF83E000BF00BFFFF78C
:102180008FFF804600BF00BFD348006820F4803036
:10219000D149086000BF00BF4046FFF785FF00BF80
:1021A00000BF6EE000BF00BFFFF77AFF804600BFB0
:1021B00000BFC948006820F40030C749086000BF6C
:1021C00000BF4046FFF770FF00BF00BF59E000BFEF
:1021D00000BFFFF765FF804600BF00BFBE48006834
:1021E00020F48020BC49086000BF00BF4046FFF7D4
:1021F0005BFF00BF00BF44E000BF00BFFFF750FF20
:10220000804600BF00BF4FF0E020006920F00100D1
:102210004FF0E021086100BF00BF4046FFF744FFD8
:1022200000BF00BF2DE04FF0E0204068401C1021AF
:1022300001EB4010C6B2B44222DAA4F11000C1177B
:1022400000EBD161C1F34715C11700EBD161491112
:10225000A0EB4111CFB200BF00BFFFF721FF8046C6
:1022600000BF00BF0120B840A90001F1E021C1F882
:10227000800100BF00BF4046FFF716FF00BF00BF50
:1022800000BF00BFBDE8F0812DE9F04104464FF0EA
:102290000008102C6BD2DFE804F0080E0F10142990
:1022A0003E090A0B0C11120D135300BF00BF00BFF3
:1022B00000BF00BF89E000BF00BF00BF00BF00BF7C
:1022C00083E000BF00BFFFF7EBFE804600BF00BF0A
:1022D0008148006840F480307F49086000BF00BF3B
:1022E0004046FFF7E1FE00BF00BF6EE000BF00BF49
:1022F000FFF7D6FE804600BF00BF7748006840F475
:1023000000307549086000BF00BF4046FFF7CCFEB3
:1023100000BF00BF59E000BF00BFFFF7C1FE80460D
:1023200000BF00BF6C48006840F480206A49086024
:1023300000BF00BF4046FFF7B7FE00BF00BF44E04C
:1023400000BF00BFFFF7ACFE804600BF00BF4FF0EC
:10235000E020006940F001004FF0E021086100BF7B
:1023600000BF4046FFF7A0FE00BF00BF2DE04FF0CA
:10237000E0204068401C102101EB4010C7B2BC4275
:1023800022DAA4F11000C11700EBD161C1F34715A7
:10239000C11700EBD1614911A0EB4111CEB200BFD2
:1023A00000BFFFF77DFE804600BF00BF0120B040A8
:1023B000A90001F1E021C1F8000100BF00BF4046C3
:1023C000FFF772FE00BF00BF00BF00BFBDE8F08195
:1023D0002DE9F04104464FF00008102C19D2DFE837
:1023E00004F0080E0F10111516090A0B0C12130D2C
:1023F000141700BF00BF00BF00BF00BF37E000BF21
:1024000000BF00BF00BF00BF00BF00BF00BF00BFD4
:102410002DE04FF0E0204068401C102101EB4010FF
:10242000C7B2BC4222DAA4F11000C11700EBD1619F
:10243000C1F34715C11700EBD1614911A0EB411160
:10244000CEB200BF00BFFFF72BFE804600BF00BF2B
:102450000120B040A90001F1E021C1F8800200BFD5
:1024600000BF4046FFF720FE00BF00BF00BF00BF17
:10247000BDE8F0812DE9F04706460D464FF0000A11
:10248000102E73D2DFE806F0080E0F10112F450949
:102490000A0B0C5B730D89A000BF00BF00BF00BF1B
:1024A00000BFE5E000BF00BFE2E000BF00BFFFF7F4
:1024B000F7FD824600BF00BF07480C38046824F0CF
:1024C000FF042C43046000BF00BF504606E000003C
:1024D000FFFF0F20FFFF0F4024ED00E0FFF7E4FDBA
:1024E00000BF00BFC4E000BF00BFFFF7D9FD8246B8
:1024F00000BF00BFCC48046824F47F4444EA0524AC
:10250000046000BF00BF5046FFF7CEFD00BF00BF14
:10251000AEE000BF00BFFFF7C3FD824600BF00BFB3
:10252000C148046824F47F0444EA0544046000BF01
:1025300000BF5046FFF7B8FD00BF00BF98E000BFE6
:1025400000BFFFF7ADFD824600BF00BFB648001DCB
:10255000046824F07F4444EA0564046000BF00BFBF
:102560005046FFF7A1FD00BF00BF81E043E000BF80
:1025700000BFFFF795FD824600BF00BFAA480830A4
:10258000046824F0FF042C43046000BF00BF5046E1
:10259000FFF78AFD00BF00BF6AE000BF00BFFFF782
:1025A0007FFD824600BF00BF9F480830046824F4C6
:1025B0007F0444EA0544046000BF00BF5046FFF7B3
:1025C00073FD00BF00BF53E000BF00BFFFF768FD11
:1025D000824600BF00BF94480830046824F07F445E
:1025E00044EA0564046000BF00BF5046FFF75CFD8D
:1025F00000BF00BF3CE04FF0E0204068401C1021CD
:1026000001EB401000F0FF094E4530DAA6F1100052
:10261000C11700EB9171C1F38707C11700EB9171EE
:102620008910A0EB810101F0FF0800BF00BFFFF798
:1026300037FD824600BF00BFB80000F1E020D0F8AF
:1026400000444FEAC801FF20884084434FEAC80194
:1026500005FA01F00443B80000F1E020C0F800449E
:1026600000BF00BF5046FFF71FFD00BF00BF00BF07
:1026700000BFBDE8F0872DE9F04706464FF0000A9D
:10268000102E70D2DFE806F0080F1215182A3D0947
:102690000A0B0C495C0D708400BF00BF00BF00BF77
:1026A00000BF624CBCE06FF00204B9E06FF00104BF
:1026B000B6E04FF0FF34B3E000BF00BFFFF7F0FC1F
:1026C000824600BF00BF58480568ECB200BF00BF9B
:1026D0005046FFF7E9FC00BF00BFA1E000BF00BF0C
:1026E000FFF7DEFC824600BF00BF4F480568C5F318
:1026F000072400BF00BF5046FFF7D6FC00BF00BF55
:102700008EE000BF00BFFFF7CBFC824600BF00BFDA
:1027100045480568C5F3074482E000BF00BFFFF7E6
:10272000BFFC824600BF00BF3F48001D05682C0E5D
:1027300000BF00BF5046FFF7B7FC00BF00BF6FE00F
:1027400000BF00BFFFF7ACFC824600BF00BF3648A9
:1027500008300568ECB200BF00BF5046FFF7A4FC8C
:1027600000BF00BF5CE026E000BF00BFFFF798FCA1
:10277000824600BF00BF2C4808300568C5F30744F7
:1027800000BF00BF5046FFF78FFC00BF00BF47E00F
:1027900000BF00BFFFF784FC824600BF00BF224895
:1027A000083005682C0E00BF00BF5046FFF77CFCC8
:1027B00000BF00BF34E04FF0E0204068401C102113
:1027C00001EB401000F0FF094E4527DAA6F110009A
:1027D000C11700EB9171C1F38707C11700EB91712D
:1027E0008910A0EB810101F0FF0800BF00BFFFF7D7
:1027F00057FC824600BF00BFB80000F1E020D0F8CF
:10280000005400BF00BF5046FFF74EFC00BF00BFA2
:102810004FEAC80025FA00F0C4B200E0034C00BF44
:1028200000BF2046BDE8F08718ED00E00080FFFF04
:1028300010B5002400BF00BFFFF732FC044600BF04
:1028400000BF1021A14800F0CFFB00BF00BF204611
:10285000FFF72AFC00BF00BF10BD10B5FFF7E8FF6F
:1028600010BD10B500209A49086002F0AFFA10BD03
:1028700010B5FFF7F6FFFFF7F0FF10BD00BFFEE752
:1028800070B505460C46002614B900BFFFF7F6FFE9
:1028900015B90A20208070BD00BF00BFFFF700FC03
:1028A000064600BF00BF10228849284601F0CAFA38
:1028B00000BF00BF3046FFF7F7FB00BF00BF00209E
:1028C000208000BFE7E72DE9F04105460C460027D0
:1028D00014B900BFFFF7D2FF1DB90A202080BDE860
:1028E000F0811021284601F095FA0646102E15D2E7
:1028F00000BF00BFFFF7D4FB074600BF00BF102298
:102900002946724801F09EFA00BF00BF3846FFF723
:10291000CBFB00BF00BF0020208002E04FF47A70A4
:10292000208000BFDBE710B502F066FA04462046BF
:1029300010BD704700B5014611B900BFFFF79EFFFB
:10294000634A106808B1002201E04FF4FA620A807D
:1029500000BD5F490860704770B505462846FFF71F
:10296000AAFB0446183C204670BD70B505462846B3
:10297000FFF7A1FB0446103C204670BD70B505462C
:102980002846FFF798FB044600BF204670BD30B5CF
:1029900002460B460024D2F1FF359C4126D24FF669
:1029A000FF74D2F1FF359C410FD26FF07F44D2F11A
:1029B000FF359C4103D2190E464C605C44E0190C73
:1029C000444C645C04F108003EE0FF24D2F1FF3582
:1029D0009C4105D2190A3F4C645C04F1100033E0BD
:1029E00019463C4C645C04F118002DE04FF6FF756D
:1029F0000024AD1A9C4115D26FF07F450024AD1A1A
:102A00009C4107D2140E44EA0321324C645C04F169
:102A1000200019E0140C44EA03412E4C645C04F1DC
:102A2000280011E00024D2F1FF059C4107D2140ACE
:102A300044EA0361274C645C04F1300004E0114671
:102A4000244C645C04F1380030BD70B504460CB908
:102A5000082070BD2046FFF731FB05462846F8E701
:102A600070B504460CB9102070BD2046FFF726FB58
:102A700005462846F8E770B504460CB9202070BD1D
:102A80002046FFF71BFB05462846F8E72DE9F043F3
:102A900004460D46002184EA01006940084302D142
:102AA0004020BDE8F083E243E843521C40F10001BE
:102AB00002EA040601EA050730463946FFF767FFD8
:102AC0008046C8F13F094846EBE700006C0600204D
:102AD0000000002030AB0000002800D17047002922
:102AE00000D17047002A00D170472DE9F81F00F08F
:102AF000030301F00304A34211D1C3F1040303F063
:102B00000303012B1DD3012A00D2F2E011F8014B7F
:102B100000F8014BA3F10103A2F10102F1E700F07B
:102B2000010301F00104A34200D094E0012B44D33F
:102B300011F8014B00F8014BA3F10103A2F10102CE
:102B4000F4E7B2F5B47F26D3B1E8F81FA0E8F81F88
:102B5000B1E8F81FA0E8F81FB1E8F81FA0E8F81FD7
:102B6000B1E8F81FA0E8F81FB1E8F81FA0E8F81FC7
:102B7000B1E8F81FA0E8F81FB1E8F81FA0E8F81FB7
:102B8000B1E8F81FA0E8F81FB1E8F81FA0E8F81FA7
:102B9000A2F5B472D5E7282A06D3B1E8F81FA0E859
:102BA000F81FA2F12802F6E7042A06D351F8043BE5
:102BB00040F8043BA2F10402F6E7202A42D331F8A0
:102BC000023B20F8023B31F8023B20F8023B31F88F
:102BD000023B20F8023B31F8023B20F8023B31F87F
:102BE000023B20F8023B31F8023B20F8023B31F86F
:102BF000023B20F8023B31F8023B20F8023B31F85F
:102C0000023B20F8023B31F8023B20F8023B31F84E
:102C1000023B20F8023B31F8023B20F8023B31F83E
:102C2000023B20F8023B31F8023B20F8023B31F82E
:102C3000023B20F8023B31F8023B20F8023BA2F1B4
:102C40002002BAE7022A06D331F8023B20F8023B01
:102C5000A2F10202F6E7102A42D311F8013B00F874
:102C6000013B11F8013B00F8013B11F8013B00F872
:102C7000013B11F8013B00F8013B11F8013B00F862
:102C8000013B11F8013B00F8013B11F8013B00F852
:102C9000013B11F8013B00F8013B11F8013B00F842
:102CA000013B11F8013B00F8013B11F8013B00F832
:102CB000013B11F8013B00F8013B11F8013B00F822
:102CC000013B11F8013B00F8013B11F8013B00F812
:102CD000013B11F8013B00F8013BA2F11002BAE7F9
:102CE000012A06D311F8013B00F8013BA2F10102D1
:102CF000F6E7BDE8F81F70470146412903DB5A2972
:102D000001DC012200E00022012A08D0612903DB56
:102D10007A2901DC012200E00022012A01D10122EE
:102D200000E00022104670470146412903DB5A2982
:102D300001DC012200E00022012A08D0612903DB26
:102D40007A2901DC012200E00022012A01D10122BE
:102D500000E00022012A08D0302903DB392901DCF8
:102D6000012200E00022012A01D1012200E000221C
:102D7000104670470146612903DB7A2901DC0122F4
:102D800000E00022104670470146412903DB5A2922
:102D900001DC012200E00022104670470146302984
:102DA00003DB392901DC012200E0002210467047D4
:102DB0000146302903DB372901DC012200E0002233
:102DC000104670470146302901DB392907DD4129CA
:102DD00001DB462903DD612903DB662901DC0122D1
:102DE00000E00022104670470146202901D0092941
:102DF00001D1012200E0002210467047014620293F
:102E000009D00D2907D00A2905D00C2903D009299A
:102E100001D00B2901D1012200E0002210467047A9
:102E20000146202903DB7E2901DC012200E000228B
:102E3000104670470146212903DB7E2901DC01226F
:102E400000E00022104670470146202903DB7E295E
:102E500001DC012200E00022012A35D1202909D01D
:102E60000D2907D00A2905D00C2903D0092901D042
:102E70000B2901D1012200E000222ABB412903DBFA
:102E80005A2901DC012200E00022012A08D0612930
:102E900003DB7A2901DC012200E00022012A01D1B2
:102EA000012200E00022012A08D0302903DB392961
:102EB00001DC012200E00022012A01D1012200E010
:102EC00000220AB9012200E00022104670470146A4
:102ED0004AB2002A01DB1F2901DD7F2901D101222D
:102EE00000E00022104670470146412903DB5A29C1
:102EF00001DC012200E00022012A02D101F12002BE
:102F000000E00A46D0B270470146612903DB7A2906
:102F100001DC012200E00022012A02D1A1F12002FD
:102F200000E00A46D0B27047F0B504460B46204692
:102F3000FFF7EAFF05461846FFF7E6FF0646B542EB
:102F400001D1012000E0002007463846F0BD000016
:102F5000FD48FE4901600146416000218160C16079
:102F6000016141618161C16101620163C1624162CC
:102F7000F7498163C1634FF4806101644164014694
:102F8000F44A116070472DE9F04103460C4617469C
:102F90000FB9BDE8F08103B9FBE70025002202E08C
:102FA0002D022543521C042AFAD3384603F0030CA1
:102FB0001946BCF1000F08D0624603E001F8014B4E
:102FC000401E521C08B1042AF8D30E4601E020C668
:102FD000001F0428FBD2314602E001F8014B401EDD
:102FE0000028FAD100BFD4E730B505460C4622468A
:102FF00000212846FFF7C7FF30BD2DE9F04F85B00F
:10300000074688469146B9F1000F02D105B0BDE8E8
:10301000F08F07B9FAE7B8F1000F00D1F6E746469E
:103020003D46AE4205D94A4641463846FFF754FD73
:10303000ECE74C463819451E08EB0400461EA81B59
:1030400004900498042834D305F00300029006F09D
:1030500003010191DDE90110884201D1012000E066
:10306000002000900098012823D10298032810D056
:10307000029840B2039008E016F8010905F801092A
:10308000641E0398401E40B2039014B103980028B8
:10309000F2DAA5F1030AA6F1030B04E05BF80409D8
:1030A0004AF80409241F042CF8D20AF103050BF195
:1030B000030604E016F8010905F80109641E002C56
:1030C000F8D100BFA2E72DE9F84F804689461546A2
:1030D00015B90120BDE8F88FB8F1000F01D100202B
:1030E000F8E7B9F1000F01D10020F3E701242946E8
:1030F00008EB050209EB050302F0030C03F0030BD8
:10310000DC4501D1012000E000200090009801285A
:1031100029D1BCF1000F12D0E2460AE0521E5B1E1C
:10312000107893F800E0704500D00024491EAAF101
:10313000010A012C03D111B1BAF1000FEED1012C1B
:1031400011D116461F4608E0361F3F1F3068D7F8DA
:1031500000E0704500D00024091F012C01D1042992
:10316000F2D232463B4608E0521E5B1E107893F8BE
:1031700000E0704500D00024491E012C01D1002937
:10318000F2D12046A6E7F0B503460D461646DA6BA7
:10319000B2FBF6F006FB102CBCF1000F02D0A6EB40
:1031A0000C0400E000246119586C884201D2002010
:1031B000F0BDA14201D3A94201D20020F8E757187F
:1031C000974201D20020F3E72244DF63586C401A93
:1031D00058641046ECE72DE9F04F81468C461C46BA
:1031E000B9FBF4F004FB109BBBF1000F02D0A4EB81
:1031F0000B0600E00026B2FBF4F004FB102BBBF141
:10320000000F02D0A4EB0B0300E00023D018ACF1B8
:10321000010E00FB0E60871806EB0208B04501D3D3
:10322000904502D20020BDE8F08FBCF1010F22D9F9
:10323000D5189D4201D3954201D20020F3E7ACF1AD
:10324000010000FB05F1A94203D3994201D3914249
:1032500001D20020E7E701EB020A8A4501D392453B
:1032600001D20020DFE7474503D38F4201D3574502
:1032700001D20020D7E73846D5E72DE9FE4F0746B3
:10328000884615461C46002000901CB900BFFFF779
:10329000F5FA00BF0DB901AD00BF002028602FB9BD
:1032A00042F2747020800020BDE8FE8FB8F1000F5C
:1032B00004D142F2757020800020F5E7DFF8889095
:1032C00000BF00BFFEF7ECFE009000BF00BFD9F8C2
:1032D0003C000290D9F844B043463A460121029896
:1032E000FFF779FF064666B900BF00BF0098FEF7FA
:1032F000DBFE00BF00BF2F6042F2E37020800020A1
:10330000D2E75E450ED900BF00BF0098FEF7CCFEA5
:1033100000BF00BFA6EB0B00286042F2E2702080E5
:103320000020C1E7424639464846FFF72CFF824657
:10333000BAF1000F15D100BF00BF0098FEF7B4FE30
:1033400000BF00BF2E6007E07C06002048454150CA
:10335000C40600200400002042F2E2702080002019
:10336000A2E700BF00BF0098FEF79EFE00BF00BFAF
:1033700042F210702080504696E72DE9FC5F064629
:103380000D461446002000901CB900BFFFF776FAE6
:1033900000BF2DB942F2757020800020BDE8FC9F6F
:1033A000B5F5805F04D942F2757020800020F5E702
:1033B00026B942F2117020800020EFE700BF00BF65
:1033C000FEF76EFE009000BF00BFFE493068084463
:1033D00040B1FD49084418B1FC49084408B900BF90
:1033E0000CE000BF00BF00BF0098FEF75DFE00BF0D
:1033F00000BF42F2887020800020CFE700BFD6F8DF
:103400000490D9F8380008B1484600E0F0488246F8
:10341000DAF84470DAF83CB000BF00BF0098FEF75D
:1034200043FE00BF00BF012D0DD9BBFBF5F005FB2E
:1034300010B8B8F1000F02D0A5EB080000E00020A2
:10344000019001983F1A42F2107020803846A5E79B
:1034500070B504460D462A462146DD48FFF78DFF2C
:103460000646304670BD70B504460D461DB900BF16
:10347000FFF704FA00BF1CB942F21170288070BD3A
:10348000D0484042206000206060A060E060206181
:103490006061A061E0612062A06260632063E0621D
:1034A0006062A063E0632064606442F21070288070
:1034B00000BFE4E72DE9FF4F91B00446DDE9209518
:1034C000002000901DB900BFFFF7D8F900BFB9F187
:1034D000000F02D10DF1100900BF0020C9F8000053
:1034E00029462046FFF7BFFF288842F21071884224
:1034F00002D015B0BDE8F08F129828B1139818B912
:1035000042F27E702880F4E7149818B942F2927063
:103510002880EEE71E9818B942F293702880E8E7F9
:103520001F9818B942F294702880E2E7A948006811
:1035300018B942F2E7702880DBE7A54810904FF0F9
:10354000000A00BF00BFFEF7ABFD009000BF00BF48
:10355000129800285BD1109E109E0E96109E374642
:10356000109EF06B0B9004231A4614990B98FFF7EA
:1035700032FE0390039850B900BF00BF0098FEF7D9
:1035800093FD00BF00BF42F2E3702880B1E70399CA
:103590000B9808440A90DDE91E2314990A98FFF756
:1035A0001AFE8346BBF1000F0AD100BF00BF00988E
:1035B000FEF77AFD00BF00BF42F2E370288098E773
:1035C000039800EB0B0A0398824501D3DA450AD22F
:1035D00000BF00BF0098FEF767FD00BF00BF42F2CA
:1035E000E370288085E71098D0F84480C2457DD9E3
:1035F00000BF00BF0098FEF757FD00BF00BFAAEB59
:103600000800C9F8000042F2E270288071E71298C1
:103610000990DDE912010844401E0890DDE9081018
:1036200081420AD200BF00BF0098FEF73DFD00BFF7
:1036300000BF42F2977028805BE7002600200E90C2
:10364000644807683AE0B96B1298814205D1396C39
:103650001398814201D13E4632E0B86B0790396C35
:10366000B86B0844401E0690DDE90701814200D294
:1036700026E007990998884203D8DDE907108842B7
:103680000FD207990998884203D30699089888426F
:1036900007D90699099888420ED806990898884251
:1036A0000AD300BF00BF0098FEF7FEFC00BF00BFBA
:1036B00042F27F7028801CE70E97FF68002FC2D16E
:1036C00000BF46B926461298A0631298E06313988B
:1036D0002064139860641098C06B0B9004231A4602
:1036E00014990B98FFF777FD039000E04CE00398E6
:1036F00050B900BF00BF0098FEF7D6FC00BF00BF66
:1037000042F2E3702880F4E61098D0F844800398E1
:1037100040450FD900BF00BF0098FEF7C5FC00BFB1
:1037200000BF0398A0EB0800C9F8000042F2E27065
:103730002880DEE6F06B0A90DDE91E2314990A98D2
:10374000FFF749FD8346BBF1000F0AD100BF00BF60
:103750000098FEF7A9FC00BF00BF42F2D970288094
:10376000C7E6D6F84480C3450ED900BF00BF009815
:10377000FEF79AFC00BF00BFABEB0800C9F80000E1
:1037800042F2D8702880B4E6149880000290042297
:1037900002991098FFF7F7FC0D900D9878BB1098E0
:1037A000D0F8448000BF00BF0098FEF77DFC00BF4A
:1037B00000BF129898B9C2450ED9AAEB0800C9F803
:1037C000000018E0B2B0B1BAFEFFFEF8080A0EFC25
:1037D0007C06002004000020C9F800A00BE002983D
:1037E000404505D90298A0EB0800C9F8000002E0A6
:1037F0000298C9F8000042F2E270288079E6FFE7FB
:103800000020019032E03046DDE91E12FFF7BBFCDC
:103810000C900C9810BBF06B0A90D6F8448000BF57
:1038200000BF0098FEF740FC00BF00BF019914984C
:10383000401A0590DDE91E2305990A98FFF7CBFC95
:103840008246C24504D9AAEB0800C9F8000001E08D
:10385000C9F800A042F2D87028804AE6019ADDE952
:103860000C0141F822000198401C01901499019824
:103870008842C8D3A6420CD10E98A060E7600E988B
:1038800010B10E98C46001E0FE4804605FB1BC60F6
:1038900009E070690F9026610F98606174610F985C
:1038A00008B10F980461F848206066600A98A0612A
:1038B0000A985844401EE0610D982062C4F828B070
:1038C0001F9860631E9820631498E06214986062E9
:1038D00000BF00BF0098FEF7E7FB00BF00BF42F249
:1038E0001070288000BF04E62DE9F04105460C4623
:1038F00000271CB900BFFEF7C1FF00BF2DB942F27F
:10390000117020800020BDE8F08100BF00BFFEF7ED
:10391000C7FB074600BF00BFDC492868084440B128
:10392000DB49084418B1DB49084408B902E00DE05E
:1039300000BF00BF00BF00BF3846FEF7B5FB00BFA9
:1039400000BF42F2887020800020DCE700BF6E6A72
:1039500000BF00BF3846FEF7A7FB00BF00BF42F222
:10396000107020803046CEE72DE9F04104460E4627
:1039700015464FF000081DB900BFFEF77FFF00BFDE
:103980002CB942F2117028800020BDE8F08126B9E0
:1039900042F2937028800020F7E700BF00BFFEF7D7
:1039A0007FFB804600BF00BFB749206888420BD02C
:1039B00000BF00BF4046FEF777FB00BF00BF42F2EA
:1039C000887028800020E0E7206BB0420BD200BF57
:1039D00000BF4046FEF768FB00BF00BF42F2937095
:1039E00028800020D1E7606A58B900BF00BF404678
:1039F000FEF75AFB00BF00BF42F2DE7028800020B5
:103A0000C3E7E16A606A88420BD900BF00BF404645
:103A1000FEF74AFB00BF00BF42F2957028800020ED
:103A2000B3E7606A401E6062D4E9080150F8217073
:103A300000BF00BF4046FEF737FB00BF00BF42F2A9
:103A4000107028803846A0E72DE9F04704460F465D
:103A500015464FF000091DB900BFFEF70FFF00BF6C
:103A60002CB942F2117028800020BDE8F08700BF19
:103A700000BFFEF715FB814600BF00BF82492068EA
:103A800088420BD000BF00BF4846FEF70DFB00BFC9
:103A900000BF42F2887028800020E6E7E16A606A91
:103AA00088420BD300BF00BF4846FEF7FDFA00BFB7
:103AB00000BF42F2957028800020D6E7E06AC01B64
:103AC000461EE06AB0420BD800BF00BF4846FEF772
:103AD000EBFA00BF00BF42F2957028800020C4E7D7
:103AE000606AB0420BD900BF00BF4846FEF7DCFA5F
:103AF00000BF00BF42F2957028800020B5E7206A21
:103B000050F8268000BF00BF4846FEF7CDFA00BF40
:103B100000BF42F2107028804046A6E72DE9F04F22
:103B200002460C469569D2F81CB0AC4201D35C4504
:103B300002D90020BDE8F08F536BB5FBF3F003FB17
:103B4000105111B1A3EB010C01E04FF0000C176B09
:103B5000B7FBF3F003FB107109B15E1A00E0002619
:103B600005EB0C08A4EB080A07EB0609BAFBF9F011
:103B700009FB10A008B9012000E00020864670462D
:103B8000D8E72DE9F04704460F4615464FF0000AE6
:103B90001DB900BFFEF772FE00BF24B942F21170DA
:103BA0002880BDE8F0871FB942F211702880F8E73D
:103BB00000BF00BFFEF774FA824600BF00BF324963
:103BC000206888420AD000BF00BF5046FEF76CFA5A
:103BD00000BF00BF42F288702880E2E739462046E5
:103BE000FFF79CFF8046B8F1010F0AD000BF00BF6D
:103BF0005046FEF759FA00BF00BF42F29770288086
:103C0000CFE7002610E0206A50F82600B8420AD11B
:103C100000BF00BF5046FEF747FA00BF00BF42F2A8
:103C200098702880BDE7761C606AB042EBD8E16AE4
:103C3000606A88420AD300BF00BF5046FEF734FADC
:103C400000BF00BF42F2DD702880AAE74FF00008F5
:103C5000666A08E0206A50F82690B94502D14FF014
:103C6000010803E0761CE06AB042F3D800BFB8F167
:103C7000010F11D1D4E9080150F82100216A41F85F
:103C8000260014E004000020504F4F4CB2B0B1BAEF
:103C9000FEFFFEF8080A0EFC00BF00BF5046FEF70C
:103CA00003FA00BF00BF42F28870288079E7D4E9A8
:103CB000080140F82170606A401C606200BF00BFCC
:103CC0005046FEF7F1F900BF00BF42F210702880A5
:103CD00000BF66E72DE9F84F04460F461546002061
:103CE00000904FF0FF3B1DB900BFFEF7C7FD00BFBE
:103CF0002CB942F2117028805846BDE8F88F27B9D8
:103D000042F2117028805846F7E700BF00BFFEF767
:103D1000C7F9009000BF00BF3D49206888420BD022
:103D200000BF00BF0098FEF7BFF900BF00BF42F21E
:103D3000887028805846E0E739462046FFF7EEFEB7
:103D40008046B8F1010F0BD000BF00BF0098FEF70E
:103D5000ABF900BF00BF42F2977028805846CCE70D
:103D6000002611E0206A50F82600B8420BD100BFAF
:103D700000BF0098FEF798F900BF00BF42F29870AC
:103D800028805846B9E7761C606AB042EAD8E16AF2
:103D9000606A88420BD300BF00BF0098FEF784F929
:103DA00000BF00BF42F2DD7028805846A5E74FF003
:103DB0000008666A08E0206A50F82690B94502D1EA
:103DC0004FF0010803E0761CE06AB042F3D800BF70
:103DD000B8F1010F0FD1E06A401EA0EB060A00BF48
:103DE00000BF0098FEF760F900BF00BF42F21070FC
:103DF0002880504681E700BF00BF0098FEF754F9C5
:103E000000BF00BF42F288702880584675E7000066
:103E1000504F4F4C10B502460B461146002001E0B2
:103E2000491C401C19B10C780CB19842F8D310BD54
:103E300030B504464FF0FF312046FFF7EBFF054653
:103E4000284630BD70B504460D4616460CB9002014
:103E500070BD0DB90020FBE721462A46002304E08F
:103E600010780870491C521C5B1C21B11AB11078E3
:103E700008B1B342F4D301B10AB90020E8E7B34274
:103E800001D2002008702046E2E770B504460D46D6
:103E90004FF0FF3229462046FFF7D4FF0646304652
:103EA00070BD70B503460C4615460BB9002070BDB9
:103EB0000CB90020FBE70DB91846F8E7194600E0F9
:103EC000491C11B108780028FAD109B90020EEE7A1
:103ED0002246002604E010780870491C521C761C0B
:103EE00021B11AB1107808B1AE42F4D301B10AB9C8
:103EF0000020DCE7002008701846D8E770B50446BB
:103F00000D464FF0FF3229462046FFF7CAFF06460E
:103F1000304670BD2DE9F04305460B469446BCF192
:103F2000000F02D10020BDE8F08335B90BB90020A5
:103F3000F9E7187842421046F5E713B92A78104697
:103F4000F1E729461C460F4626467F1C761C4FF09B
:103F5000000805E0491C641C7F1C761C08F1010860
:103F6000087894F80090484505D1087818B117B141
:103F70000EB1E045EED3E04501D10020D3E708784B
:103F800094F80090484505D0087894F80090A0EB8C
:103F900009020BE0087808B9002207E02FB90EB932
:103FA000002203E03078424200E03A781046BAE757
:103FB00070B504460D464FF0FF3229462046FFF704
:103FC000A9FF0646304670BD2DE9F74F82B0804606
:103FD0000E46049818B9002005B0BDE8F08FB8F17E
:103FE000000F09D10EB90020F6E73078FEF77CFF0C
:103FF00007467C422046EFE73EB998F80000FEF7FE
:1040000073FF05462C462046E6E7C146B246C84641
:10401000C3465646CDF804A0D8460BF1010B019ECD
:10402000701C0190C84699F80000FEF75DFF054638
:1040300056469AF80000FEF757FF0746002000900A
:1040400015E009F101090AF1010A0BF1010B0198D0
:10405000401C01900098401C009099F80000FEF769
:1040600043FF05469AF80000FEF73EFF0746BD42B3
:104070000BD199F8000040B1BBF1000F05D00198B9
:1040800018B1049900988842DBD3049900988842BB
:1040900001D10020A0E7BD4201D0EC1B16E00DB914
:1040A000002413E0BBF1000F0AD1019808B90024E5
:1040B0000CE001990878FEF717FF07467C4205E0FF
:1040C0009BF80000FEF710FF05462C46204683E7CC
:1040D00070B504460D464FF0FF3229462046FFF7E3
:1040E00073FF0646304670BD30B504460B46154694
:1040F0000CB9002030BD0BB90020FBE7214600229F
:1041000001E0491C521C31B1087820B10878A8425E
:1041100001D09A42F5D309B90020EBE79A4201D3C6
:104120000020E7E70878A84201D00020E2E708462F
:10413000E0E770B505460C4622464FF0FF312846B1
:10414000FFF7D2FF0646304670BD2DE9F043054625
:104150000E46174615B90020BDE8F0830EB90020C1
:10416000FAE72C46A6F1010949462046FFF752FE20
:10417000804644440CB90020EEE700E0641EAC42E7
:1041800002D02078B842F9D12078B84201D000207E
:10419000E2E72046E0E770B505460C4622464FF0C0
:1041A000FF312846FFF7D1FF0646304670BD70B597
:1041B00004460D4616460CB9002070BD0BB9002010
:1041C000FBE721461A4605E00878A84200D10E70A8
:1041D000491C521E19B1087808B1002AF4D12046B2
:1041E000EBE7F0B504460D4616464FF0FF33324676
:1041F00029462046FFF7DBFF07463846F0BD2DE98C
:10420000FF4F06460F4615461EB9002004B0BDE814
:10421000F08F0FB90020F9E70DB90020F6E7681C10
:1042200000B101E04FF0FF30039029463046FFF720
:10423000F1FD804638460399FFF7ECFD04460CB9C2
:104240003046E3E7444501D90020DFE706EB080BE1
:10425000BBF1000F01D10020D8E707EB040BBBF145
:10426000000F01D10020D1E7A8EB040002904FF02D
:1042700000090020019000BF06EB090000902246D3
:1042800039460098FFF746FE8246BAF1000F01D189
:10429000012000E00020019009F10109019810B906
:1042A00002988145E8D9BAF1000F01D00020ADE7AE
:1042B0000098ABE770B504460D464FF0FF32294633
:1042C0002046FFF79CFF0646304670BD2DE9FF4FA4
:1042D0008DB00F4615461A9E1D9818B9002011B0D2
:1042E000BDE8F08F002003900490012F01DA012037
:1042F0000390022D01D3242D01D90120039096B300
:104300003046FEF78DFD02900298012802D0012070
:10431000039028E0302E26D0A6F13000C0B20790DE
:104320001B98012804D0A6F14100C0B2069003E01A
:10433000A6F16100C0B206900A2D02D80798A842E3
:1043400009DB0A2D09D907980A2804D3A5F10A0028
:104350000699884201D9012000E0002005900598C7
:10436000012800D103901D9C0398002846D1DDF858
:1043700034A0DDF834A0CDF830A001200B9007E088
:104380000B98401CC0B20B900C98B0FBF5F00C9051
:104390000C98A842F4D21098012800D100E0002027
:1043A00009900B9909980844B84225DC0020019037
:1043B0000B98B84201DA0B9800E038460A903EB1FB
:1043C000B8460A98391A0998081AC0B2089006E047
:1043D000DDE90910084400F0FF0800200890089863
:1043E000002806DD302E01D1012000E000200490DD
:1043F00004E00020049001E001200390039800B144
:10440000B84644441C9808B100202070641E4FF048
:10441000000941E00398A8BBBAF1000F02D1B9F13D
:10442000000F1CD1BAFBF5F005FB10A000F0FF0B4C
:10443000BBF10A0F04D20BF1300004F801090BE0C4
:104440001B98012804D00BF1370004F8010903E0A0
:104450000BF1570004F80109BAFBF5FA1AE01098BD
:10446000012810D1049808B9019828B1049850B1D6
:10447000A8F10100484506D12D2004F801090120CA
:10448000019007E003E02EB104F8016902E03F204B
:1044900004F8010909F10109C145BBD3039808B12A
:1044A00000201CE71D981AE72DE9FF5F05460E4620
:1044B00017461C46DDE90F9ADDF8388000233A469E
:1044C000314628468DE81007FFF700FF834658461F
:1044D00004B0BDE8F09F2DE9FF4F85B00446894642
:1044E0001F46DDE913AB002C02DA6542012601E02C
:1044F0002546002612983346CDE902ABCDE900707F
:1045000049462846079AFFF7E1FE8046404609B033
:10451000BDE8F08F2DE9FF4F8BB006468946154662
:10452000B9F1000F02D10DF1240900BFC9F80060F4
:10453000189810B907A8189000BF002118980170AA
:104540001EB900200FB0BDE8F08F012D01D0242D41
:1045500001D90020F6E734462078FEF74FFC03909F
:1045600004E0641C2078FEF749FC039003980128BE
:10457000F7D020782B2802D02D280BD103E0641C23
:104580004FF0000B09E00E98012800D1641C4FF099
:10459000010B02E04FF0000B00BF00BF0A9425B1F1
:1045A000082D1CD0102D36D11EE02078302814D1D3
:1045B000641C2078582802D078280BD100BF102521
:1045C00067783846FEF7FEFB8246BAF1010F00D14C
:1045D000641C01E0082500BF00E00A251CE02078EB
:1045E000302800D1641C17E02078302812D1641CD8
:1045F0002078582802D078280AD100BF677838463A
:10460000FEF7E0FB8246BAF1010F00D1641C00E026
:1046100000BF00BF00E000BF00BF4FF00008002057
:104620000290019040E027783846FEF77DFB059028
:104630000598012836D13846FEF7B0FB069006985B
:10464000012804D1A7F13000C0B208900FE038462D
:10465000FEF790FB04900498012804D1A7F15700BD
:10466000C0B2089003E0A7F13700C0B208900898E4
:10467000A84214DA029880B9304850F82500404525
:1046800009D308FB05F8089880440898804504D2AF
:104690000120029001E001200290641C04E001204E
:1046A000019001E00120019001980028BBD0029800
:1046B000012801D14FF0FF380A98844202D0C9F88E
:1046C000004001E0C9F80060189880F800B040464A
:1046D00038E7F8B504460D46164600200346324634
:1046E000294600902046FFF715FF07463846F8BDDB
:1046F0002DE9FC4105460E46174601A801233A461E
:10470000314600902846FFF705FF04469DF8040057
:1047100040B9B4F1004F02D36FF0004000E02046F2
:10472000804607E0B4F1004F02D34FF0004000E0B4
:10473000604280464046BDE8FC81000034AC000089
:1047400010B500F036F800F091FA10BD704710B5C2
:104750000446702C04D204F11001C8B2FDF7F0FC3D
:1047600010BD10B5FDF798FC10BD10B50446702CB7
:1047700004D204F11001C8B2FDF786FD10BD70B57A
:1047800004460D460026702C10D200BF00BFFDF776
:1047900087FC064600BF00BFF84840F8245000BF21
:1047A00000BF3046FDF780FC00BF00BF70BD00BFFA
:1047B000FEE710B5002404E0E0B2F149FFF7DFFFA7
:1047C000641C702CF8D310BD70B50446002600BFE1
:1047D00000BFFDF765FC064600BF00BF00F0E2FE2B
:1047E00000BF00BF3046FDF75FFC00BF00BF702C6C
:1047F00004D2E24850F8245005B1A84700F0E8FE82
:1048000070BD10B50020FFF7DFFF10BD10B501200F
:10481000FFF7DAFF10BD10B50220FFF7D5FF10BD7E
:1048200010B50320FFF7D0FF10BD10B50420FFF72F
:10483000CBFF10BD10B50520FFF7C6FF10BD10B5AA
:104840000620FFF7C1FF10BD10B50720FFF7BCFF22
:1048500010BD10B50820FFF7B7FF10BD10B5092037
:10486000FFF7B2FF10BD10B50A20FFF7ADFF10BD76
:1048700010B50B20FFF7A8FF10BD10B50C20FFF7F7
:10488000A3FF10BD10B50D20FFF79EFF10BD10B5A2
:104890000E20FFF799FF10BD10B50F20FFF794FF12
:1048A00010BD10B51020FFF78FFF10BD10B51120FF
:1048B000FFF78AFF10BD10B51220FFF785FF10BD6E
:1048C00010B51320FFF780FF10BD10B51420FFF7BF
:1048D0007BFF10BD10B51520FFF776FF10BD10B59A
:1048E0001620FFF771FF10BD10B51720FFF76CFF02
:1048F00010BD10B51820FFF767FF10BD10B51920C7
:10490000FFF762FF10BD10B51A20FFF75DFF10BD65
:1049100010B51B20FFF758FF10BD10B51C20FFF786
:1049200053FF10BD10B51D20FFF74EFF10BD10B591
:104930001E20FFF749FF10BD10B51F20FFF744FFF1
:1049400010BD10B52020FFF73FFF10BD10B521208E
:10495000FFF73AFF10BD10B52220FFF735FF10BD5D
:1049600010B52320FFF730FF10BD10B52420FFF74E
:104970002BFF10BD10B52520FFF726FF10BD10B589
:104980002620FFF721FF10BD10B52720FFF71CFFE1
:1049900010BD10B52820FFF717FF10BD10B5292056
:1049A000FFF712FF10BD10B52A20FFF70DFF10BD55
:1049B00010B52B20FFF708FF10BD10B52C20FFF716
:1049C00003FF10BD10B52D20FFF7FEFE10BD10B582
:1049D0002E20FFF7F9FE10BD10B52F20FFF7F4FED3
:1049E00010BD10B53020FFF7EFFE10BD10B531201F
:1049F000FFF7EAFE10BD10B53220FFF7E5FE10BD4F
:104A000010B53320FFF7E0FE10BD10B53420FFF7DE
:104A1000DBFE10BD10B53520FFF7D6FE10BD10B57A
:104A20003620FFF7D1FE10BD10B53720FFF7CCFEC2
:104A300010BD10B53820FFF7C7FE10BD10B53920E6
:104A4000FFF7C2FE10BD10B53A20FFF7BDFE10BD46
:104A500010B53B20FFF7B8FE10BD10B53C20FFF7A6
:104A6000B3FE10BD10B53D20FFF7AEFE10BD10B572
:104A70003E20FFF7A9FE10BD10B53F20FFF7A4FEB2
:104A800010BD10B54020FFF79FFE10BD10B54120AE
:104A9000FFF79AFE10BD10B54220FFF795FE10BD3E
:104AA00010B54320FFF790FE10BD10B54420FFF76E
:104AB0008BFE10BD10B54520FFF786FE10BD10B56A
:104AC0004620FFF781FE10BD10B54720FFF77CFEA2
:104AD00010BD10B54820FFF777FE10BD10B5492076
:104AE000FFF772FE10BD10B54A20FFF76DFE10BD36
:104AF00010B54B20FFF768FE10BD10B54C20FFF736
:104B000063FE10BD10B54D20FFF75EFE10BD10B561
:104B10004E20FFF759FE10BD10B54F20FFF754FE91
:104B200010BD10B55020FFF74FFE10BD10B551203D
:104B3000FFF74AFE10BD10B55220FFF745FE10BD2D
:104B400010B55320FFF740FE10BD10B55420FFF7FD
:104B50003BFE10BD10B55520FFF736FE10BD10B559
:104B60005620FFF731FE10BD10B55720FFF72CFE81
:104B700010BD10B55820FFF727FE10BDC40A002055
:104B8000AF47000010B55920FFF71EFE10BD10B54D
:104B90005A20FFF719FE10BD10B55B20FFF714FE79
:104BA00010BD10B55C20FFF70FFE10BD10B55D20E5
:104BB000FFF70AFE10BD10B55E20FFF705FE10BD21
:104BC00010B55F20FFF700FE10BD10B56020FFF7A5
:104BD000FBFD10BD10B56120FFF7F6FD10BD10B54F
:104BE0006220FFF7F1FD10BD10B56320FFF7ECFD6B
:104BF00010BD10B56420FFF7E7FD10BD10B56520AE
:104C0000FFF7E2FD10BD10B56620FFF7DDFD10BD1A
:104C100010B56720FFF7D8FD10BD10B56820FFF76D
:104C2000D3FD10BD10B56920FFF7CEFD10BD10B546
:104C30006A20FFF7C9FD10BD10B56B20FFF7C4FD5A
:104C400010BD10B56C20FFF7BFFD10BD10B56D2075
:104C5000FFF7BAFD10BD10B56E20FFF7B5FD10BD12
:104C600010B56F20FFF7B0FD10BD00004F48C06FBA
:104C700020F01C004D49C8670846C06F40F0100086
:104C8000C8674A48C0300068494908404749C1F8E8
:104C9000C0004648C0300068464908434349C03117
:104CA000086048064149B03108604FF04C70086018
:104CB00060204149086004203C49C1F864013E4835
:104CC000A03800683A4908403849C1F8C0003A485D
:104CD000A0380068394908433449C1F8C000084683
:104CE000D0F8600140F40000C1F8600100BF324814
:104CF0000830006800F0010080F001000028F6D1C3
:104D00002A48B03000682E4908432849C1F8B0004D
:104D100070472DE9F043DFF894C0DCF8B0C0CCF365
:104D2000007CBCF1000F3ED0DFF880C0DCF860C131
:104D3000CCF38A24DFF874C0DCF860C1CCF30A033A
:104D400003EB9422DFF864C0DCF864C1CCF30425E3
:104D5000DFF858C0DCF864C10CF01F06DFF84CC067
:104D6000DCF8B0C0CCF3036111B1032904D101E038
:104D7000144902E0144900E000BF00BF01FB02F843
:104D800005F1010C06F101090CFB09FCB8FBFCF074
:104D9000DFF818C0DCF8B0C0CCF3090C0CF1010747
:104DA000B0FBF7F000E00020BDE8F08300E00F402A
:104DB00010FC10FC8100010060E10F4085018501BD
:104DC000030000900024F40040787D0110B51948DC
:104DD000006840F08070174908600020164948605C
:104DE0000846006840F001000860FFF792FF0446A3
:104DF0002046FDF7AEFD10BD0F49486870472DE90C
:104E0000F0478246FFF785FF4FF0000980460B4AC6
:104E100000234046494605F0E7F8064632460B4671
:104E20005046002105F0E0F804460D46204629468C
:104E3000BDE8F087FCED00E0001000E040420F000C
:104E40000146002002E0491C421CD0B20A78002A28
:104E5000F9D170472DE9F04105460E46144600276A
:104E6000FB48007820B1112020700020BDE8F081BF
:104E70002878012808D0022807D0032802D0042867
:104E800004D100E000BF00BF00BF03E0012020709C
:104E90000020EBE700BF03F09DF80746686930602B
:104EA0003068FFF7CDFF8046384603F097F80020C2
:104EB00020704046DAE72DE9F04105460E461446DB
:104EC0000027E348007818B112202070BDE8F08177
:104ED0002878012808D0022807D0032802D0042807
:104EE00004D100E000BF00BF00BF02E0012020703D
:104EF000ECE700BF03F06EF807466E61384603F03A
:104F00006DF80020207000BFE0E7F0B5024612F80F
:104F1000384F95785678383A0B4618680FE000F10C
:104F20000B073F5DB74300F10B0C0CF804706746AC
:104F30003F5D17B9877AAF4387721B1D1868002839
:104F4000EDD1F0BDC349C44A1278885CC349095CFD
:104F5000C04A515C01EBC001C14A1170704710B5E5
:104F6000002403F037F80446B9480078F8B9BD4882
:104F70000078E0B9FFF7E6FFBB48B949097850F877
:104F80002100BA490860B6480078B94909788842D2
:104F90000DD0B6480068C06B401CB4490968C863AE
:104FA000B4480068401CB349086003F02EF820465E
:104FB00003F014F810BD70B501460024AE4D2D6805
:104FC000EC61AD4C246821620B4618681BE0AA4CCA
:104FD000246894F8385000F10B04645DA64D2D68E8
:104FE00095F839502C43A44D2D6895F8386000F1A0
:104FF0000B05AC55847AA04D2D6895F83A502C439A
:1050000084721B1D18680028E1D19B4C246894F819
:105010003820924CA45C984D2D6895F83950AC43DB
:105020008E4DAC542C46A45C44B9934C246894F83F
:105030003A50894C2478AC43874D2C7070BD2DE9D3
:10504000FF4F83B081460E461546DDF840800020B4
:1050500000903060CA46DAF8004018E02078062850
:1050600007D2DFE800F00604050307080AE009E0BC
:1050700008E000BF00BF012088F80000002007B052
:10508000BDE8F08F00BF0AF1040ADAF80040002CF6
:10509000E4D16F48007820B1022088F80000002099
:1050A000EDE77048007820B10D2088F8000000205E
:1050B000E5E70020029001908346CA46DAF80040F6
:1050C00002F088FF009057E02078062843D2DFE8FE
:1050D00000F0421526034344208960B12089401E18
:1050E000208110C601200290002001C50198401CBB
:1050F00080B2019001E04BF0010B38E0606858B1DC
:10510000606801C50020606010C60120029001980F
:10511000401C80B2019001E04BF0020B27E0676871
:10512000F88AA8B13969081D3861086801C5B968ED
:105130003869884201D178683861F88A401EF8825F
:1051400010C6012002900198401C80B2019001E03D
:105150004BF0040B0BE000BF00BF009802F03EFFD5
:1051600000203060012088F80000019887E700BF28
:105170000AF1040ADAF80040002CA5D102980128AF
:1051800009D100203060009802F028FF002088F844
:105190000000019873E73848006890F834004BF03D
:1051A000800108433449096881F8340000203249FD
:1051B000096881F83500304906980968086348464F
:1051C000FFF7F9FE009802F009FFFFF7C8FE02F0B2
:1051D00001FF00902848006890F8350020B10128B0
:1051E00019D0022816D100E000BF23480068C46926
:1051F0002CB110C6002030600120019009E0012090
:105200001D49096881F8350049461B480068FFF7C9
:105210007CFE06E000BF494617480068FFF775FEB0
:1052200000BF00BF1448006890F8350020B1012885
:1052300042D002283FD138E02078062824D2DFE887
:1052400000F0231D1E032425002001C528E00000D6
:1052500021000020C8AC000025000020260000200E
:105260002400002022000020241700203C00002001
:1052700023000020080000203400002000BFFD486B
:105280000068406A01C50BE000BF00BF009802F053
:10529000A5FE00203060012088F800000198EEE6AD
:1052A00000BF002088F800000CE0002001C50E209F
:1052B00088F8000006E000BF002001C50A2088F839
:1052C000000000BF00BF0020EA49096881F83400EF
:1052D000E849096881F83500E6490968C861E54987
:1052E00009680862E34909684862009802F076FE9E
:1052F0000198C4E67CB5002514E06946284602F012
:105300000EF9064666B9DC4850F8254044B1012C38
:1053100006D0D4E9020100EB8100A0640198E064AA
:10532000681CC5B23F2DE8D97CBD00BF00BF02E0BC
:10533000C82002F01BFAD14800780028F8D0D048E5
:1053400000686421B0FBF1F0CD49086008460068B0
:1053500028B90020CB490870FF2002F020F902F0A4
:1053600039FE0446C648006864214843C6490860BF
:10537000204602F033FE00BF02F02CFE0446C24875
:105380000068C24908600020BF490860204602F05A
:1053900025FEBE480068BA490968B0FBF1F0C0F1CB
:1053A0006400B849087002F098FEFFF7A3FF64207C
:1053B00002F0DCF9E0E700B587B00320002180228D
:1053C000B34BCDE90132CDE903104FF6FE703E2319
:1053D000B04A0090AFF2AD0001F0B3FE06AAAEA154
:1053E0003E2002F01EF807B000BD002400BF00BF41
:1053F00002F0F0FD0446A4480068401CA249086081
:10540000204602F0EBFD02F05EFEF1E700B587B04A
:10541000032000218022A44BCDE90132CDE9031005
:105420004FF6FF703F23A14A0090AFF2410001F018
:1054300088FE06AA9EA13F2001F0F3FF07B000BD41
:1054400004E0002200F8012B4A1E91B20029F8D195
:10545000704770B54FF4C0619948FFF7F1FF002421
:1054600011E0601C85B204EB4400954901EBC003D8
:1054700005EB450001EBC006002018705E6091A0AE
:105480005861601C84B23F2CEBD304EB44008C4980
:1054900001EBC0030020187058608AA058610846CC
:1054A0008949086070BD70B54FF4F2618748FFF715
:1054B000C7FF4FF480717048FFF7C2FF002413E06C
:1054C000601CC5B204EB440000EBC4007F4901EB53
:1054D000C00305EB450000EBC50001EBC0065E61B3
:1054E00078A01865601CC4B2152CE9D304EB440005
:1054F00000EBC400754901EBC0030020586171A0A6
:10550000186500207249086070487249086070BDD3
:105510000021714A1170002004E000216F4A1154EB
:10552000411CC8B20828F8D300216D4A11706D4A99
:1055300011706D4A11604F4A1160704700206B492D
:1055400008606B4908706B4908706B4908706B49BB
:1055500008706B4908604C4908604C49086048492C
:1055600008604649087067490870704710B502F036
:1055700089FDFFF7E3FFFFF7CBFFFFF794FFFFF78E
:1055800068FF00F0CFFE00F0C0FF01F0C2FAFFF7A5
:105590003DFFFFF710FF02F075FC02F087FD02F0FF
:1055A00001FF10BD10B5002402F014FD044653485D
:1055B0000078012808D14E480078FF2804D24C48D2
:1055C0000078401C4A490870204602F007FD10BDD3
:1055D00010B5002449480078012830D102F0FAFCC7
:1055E00004464348007820B141480078401E4049B5
:1055F00008703F480078F8B93E480078E0B9FFF7F6
:10560000A1FC1D483749097850F821003649086047
:10561000344800783249097888420DD03248006811
:10562000C06B401C30490968C86335480068401C9D
:105630003349086002F0EEFC204602F0CFFC10BDBA
:1056400010B500242D480078012811D102F0C2FCC9
:1056500004462748007840B926480078FF2804D23D
:1056600024480078401C23490870204602F0B6FC0C
:1056700010BD00003400002024170020200000206E
:105680001800002014000020300000201C00002022
:10569000241300202015002075432F4F532D494916
:1056A000205374617400000024150020201700208E
:1056B00075432F4F532D49492049646C6500000004
:1056C000840C00203F0000000C0000202418002063
:1056D0004000002038000020250000202600002087
:1056E00023000020240000203C0000205400002063
:1056F00021000020220000202F0000202E0000208A
:10570000080000205000002010B50024FD4800785B
:10571000012821D102F05EFC0446FB480078C0B9A4
:10572000FA48007888B1F9480078401EF7490870B7
:105730000846007828B9204602F050FCFFF70FFC1D
:105740000AE0204602F04AFC06E0204602F046FC51
:1057500002E0204602F042FC10BD10B5E948007896
:1057600090B9FFF7EFFBEA480078EA490870EA4889
:10577000E749097850F82100E849086008460068C0
:10578000E749086002F02DFC10BD10B5002402208E
:1057900001F0ECFF02F01EFC04460020E149086025
:1057A000204602F01BFC642001F0E0FF02F012FC36
:1057B0000446DC480068DC4908600120DB490870C9
:1057C000204602F00BFC10BD70B5002602F071FD02
:1057D00002F000FC0646D6480068401CD449086028
:1057E000304602F0FBFBC7480078012853D1D1486E
:1057F000007820B1012804D0022809D103E0012556
:105800000BE0002509E001250120CA49087004E0E9
:1058100001250020C749087000BF00BF05B970BD51
:10582000C548046833E002F0D5FB0646206B50B350
:10583000206B401E2063206B28BB94F8340000F0DE
:10584000370040B114F8340F00F0C8002070012078
:105850006070343C02E0002084F8350094F8340095
:1058600000F0080078B93834A078B44909780843C2
:10587000B24908702078B249085C6178084314F88E
:105880003819AF4A50546469304602F0A7FB94F8C7
:1058900036003F28C7D100BFC1E747F21A20704742
:1058A000704710B590F8382001F10B039B5C90F81D
:1058B0003940A34301F10B04A35423469B5C23B955
:1058C0008B7A90F83A40A3438B720023C36110BDDA
:1058D0002DE9F04F05460F4690469946A87A99491A
:1058E0000E5C05F10B00805D11F800B00BEBC600FB
:1058F00000F0FF0A884850F82A4000202434E06075
:105900002760207C20EA0800207484F81190207C15
:10591000243C00F0080068B994F83A0087490978F7
:105920000843864908708648805D94F8391008431A
:105930008349885529462046FFF7B3FF206A20B1E6
:105940002046216AFFF7E1FAE5615046BDE8F08F95
:1059500010B5734A1268D061714A126892F83830F3
:1059600000F10B02D25C6E4B1B6893F839301A437E
:105970006B4B1B6893F8384000F10B031A55827A81
:10598000674B1B6893F83A301A438272644A126874
:1059900092F838106A4A525C614B1B6893F83930B0
:1059A0009A43674B5A541A46525C42B95C4A126891
:1059B00092F83A30614A12789A43604B1A7010BDDF
:1059C000014600228A72002005E0002301F10B024B
:1059D0001354421CD0B20828F7D3704705E011F8E1
:1059E000013B00F8013B531E9AB2002AF7D17047E1
:1059F0002DE9F84F05460F4690469946DDE90AAB7A
:105A00000020009002F0E6FA00904F480468002C55
:105A100077D01C3454F8080C4B490860009802F009
:105A2000DDFA44F81C7CA576002020766076606163
:105A300044F818BC44F810AC44F8148C0C9824F8C2
:105A40000C0C24F80A9C0020E077E810207705F081
:105A50000700E076217F01208840A077E17E0120C9
:105A600088406077002020606060E060A060206275
:105A7000A0626062E0622063AFF2B83060631C3CF9
:105A8000002606E0002104F1540040F82610701CA6
:105A9000C6B2002EF6D0204602F005FC02F09AFABB
:105AA00000901D4840F82540009802F097FA2046E3
:105AB00002F0FDFA02F08EFA00901F480068606163
:105AC0000020A0611C48006810B11B480068846178
:105AD000194804603834A0781849097808431749F0
:105AE000087020781649085C6178084314F8381962
:105AF000134A505415480078401C14490870009807
:105B000026E02AE02E0000202100002022000020B4
:105B10002400002023000020241700203C00002047
:105B20003400002030000020180000202000002059
:105B300054000020440000204000002025000020E8
:105B400026000020C8AC0000380000202F000020F4
:105B500002F044FA0020BDE8F88F009802F03EFA07
:105B60004220F8E72DE9F05F04460F4691461E46B5
:105B70004FF0000B2078052804D001203070002061
:105B8000BDE8F09F09F0800ABAF1000F04D029F0B7
:105B900080094FF0010801E04FF00008002030704C
:105BA00002F018FA8346B9F1000F2CD0B9F1010FB9
:105BB0003BD0B9F1020F03D0B9F1030F46D111E088
:105BC000208900EA0705BD4206D1B8F1010F05D1D1
:105BD0002089A843208101E070203070584602F0EF
:105BE000FDF93AE0208900EA070535B1B8F1010F67
:105BF00005D12089A843208101E0702030705846EB
:105C000002F0ECF929E0208927EA0005BD4206D11F
:105C1000B8F1010F05D120892843208101E07020CF
:105C20003070584602F0DAF917E0208927EA0005BB
:105C300035B1B8F1010F05D120892843208101E059
:105C400070203070584602F0C9F906E0584602F05C
:105C5000C5F900256F20307000BF00BF28468FE7D0
:105C60002DE9F04106460D460027FC48007820B19A
:105C7000102028700020BDE8F08102F0ABF9074643
:105C8000F748046884B100684068F5490860052059
:105C90002070268100206060F2A0E060384602F0AB
:105CA0009DF90020287004E0384602F097F9722030
:105CB00028702046DFE730B501464A6808682AB9EF
:105CC000CC68606028B10025456002E0106000B13A
:105CD00042608B6800259D6230BD2DE9F04106468B
:105CE00088461746B468002044F8300F24F8048C26
:105CF000207900F0DF00207167712079303C88B98D
:105D00003834A078D84909780843D74908702078F2
:105D1000D649085C6178084314F83819D34A5054BE
:105D2000012500E000253046FFF7C5FF2846BDE805
:105D3000F0812DE9F0470446894615464FF0000AE8
:105D4000C648007820B10F2028702046BDE8F087B3
:105D50002078052803D0012028702046F6E702F0BD
:105D600039F98246606808B1012700E00027B9F1DF
:105D7000000F03D0B9F1010F3DD119E08FB9B9A0DF
:105D8000E06000202070B64800686060002020813C
:105D9000B3480460504602F021F900202870002624
:105DA00005E0504602F01AF949202870264629E0FD
:105DB000D4F8048006E0022200214046FFF78DFF60
:105DC000D8F80080B8F1000FF5D1A6A0E06000205F
:105DD0002070A3480068606000202081A048046013
:105DE000504602F0FBF8012F01D1FFF7B8F8002070
:105DF0002870002606E0504602F0F0F807202870D0
:105E0000264600BF00BF3046A0E72DE9F041054619
:105E10000E46144600279148007820B111202070CA
:105E20000020BDE8F08102F0D5F807462878052863
:105E300006D0384602F0D2F8012020700020F0E7AA
:105E4000E86830603068FEF7FBFF8046384602F0B5
:105E5000C5F8002020704046E3E72DE9F0410546F3
:105E60000E46144600277D48007818B11220207095
:105E7000BDE8F08102F0AEF807462878052805D085
:105E8000384602F0ABF801202070F1E7EE603846AA
:105E900002F0A4F80020207000BFE9E7F0B5144636
:105EA000059E734F3F6897F8347047F02007DFF87E
:105EB000C0C1DCF800C08CF834700027DFF8B0C136
:105EC000DCF800C08CF83570694F3F683E63684F5E
:105ED0003F68B9620C828B74654F3F688F6047687A
:105EE0000F6000274F60C860456805B16960416078
:105EF0005F4F3F6897F838205C4FBF5CDFF870C198
:105F0000DCF800C09CF839C027EA0C07DFF85CC158
:105F10000CF802706746BF5C5FB9554F3F6897F851
:105F20003AC0514F3F7827EA0C07DFF83CC18CF8A4
:105F30000070F0BD2DE9F04F89B005460F4691463F
:105F40009A46129E002002904448007828B1022010
:105F50003070002009B0BDE8F08F4648007818B1D5
:105F60000D2030700020F5E72878052803D00120A7
:105F700030700020EEE709F0800BBBF1000F04D079
:105F800009F07F094FF0010801E04FF0000802F02E
:105F900021F80290B9F1000F4AD0B9F1010F78D081
:105FA000B9F1020F03D0B9F1030F71D120E02889B4
:105FB00000EA0704BC420FD1B8F1010F02D12889D1
:105FC000A04328812A4800688485029802F006F8D8
:105FD000002030702046BDE74B463A4604A92846CB
:105FE000CDF800A0FFF75AFF029801F0F7FF78E024
:105FF000288900EA07047CB1B8F1010F02D1288991
:10600000A04328811A4800688485029801F0E6FFC1
:106010000020307020469DE74B463A4604A92846AA
:10602000CDF800A0FFF73AFF029801F0D7FF58E043
:10603000288927EA0004BC421ED1B8F1010F02D121
:106040002889204328810A4800688485029801F045
:10605000C5FF0020307020467CE71AE021000020B8
:10606000100000203F000000250000202600002036
:1060700034000020220000204B463A4604A928465E
:10608000CDF800A0FFF70AFF029801F0A7FF28E073
:106090001FE0288927EA00047CB1B8F1010F02D182
:1060A000288920432881B34800688485029801F03C
:1060B00095FF0020307020464CE74B463A4604A935
:1060C0002846CDF800A0FFF7E9FE029801F086FF10
:1060D00007E0029801F082FF00246F203070204614
:1060E00038E700BFFEF73BFF01F074FF0290A148C4
:1060F000006890F8350020B39E48006890F835009D
:10610000039000209B49096881F8350004A8FFF737
:10611000D2FD00209749096881F83400029801F007
:106120005DFF00240398012805D0022802D10E202B
:10613000307003E000BF0A20307000BF00BF20466F
:1061400008E78C480068848DB8F1010F1ED1B9F1C1
:10615000000F0ED0B9F1010F0CD0B9F1020F03D02E
:10616000B9F1030F0AD100E000BF2889A0432881BC
:106170000BE000BF28892043288106E0029801F047
:106180002DFF6F2030700020E4E600BF029801F080
:1061900025FF002030702046DCE670B5002501F0B8
:1061A00019FF054673480068848D284601F016FFE4
:1061B000204670BD2DE9FC5F0446894692461E4686
:1061C000002000902078052804D0012030700020A5
:1061D000BDE8FC9F01F0FEFE0090BAF1000F03D075
:1061E000BAF1010F0AD104E0208920EA09002081D8
:1061F0000BE0208940EA0900208106E0009801F0C8
:10620000EDFE712030700020E2E700BF4FF0000B80
:10621000656859E0A87C50B301283BD0022802D021
:10622000032848D112E02089298A00EA0107288A38
:10623000B8420AD1002239462846FFF74EFD804673
:10624000B8F1010F01D14FF0010B3BE02089298A01
:1062500000EA010757B1002239462846FFF73DFD05
:106260008046B8F1010F01D14FF0010B2AE0288AD6
:10627000218920EA0107288AB8420AD1002239463A
:106280002846FFF72AFD8046B8F1010F01D14FF0F3
:10629000010B17E0288A218920EA010757B1002263
:1062A00039462846FFF719FD8046B8F1010F01D1A4
:1062B0004FF0010B06E0009801F090FE6F20307067
:1062C000002085E700BF2D68002DA3D1009801F0C4
:1062D00085FEBBF1010F01D1FEF741FE01F07AFE10
:1062E000009020890190009801F078FE0020307025
:1062F00001986DE72DE9F04104460D46002720780E
:10630000052804D0012028700020BDE8F08101F0AC
:1063100061FE07462689384601F060FE002028709D
:106320003046F2E72DE9F041A0211348FFF788F845
:1063300000250EE0681C86B20F4800EB051400EB48
:106340000617002020706760AFF2E820E060681C4C
:1063500085B2092DEED3084800EB0514002020700B
:106360006060AFF20030E060034804490860BDE8B7
:10637000F081000034000020841200201000002072
:106380002DE9FC5F05460F4691469A460020009095
:1063900001F020FE00906F480468006820B16D484D
:1063A000006840686B490860009801F017FE2CB93E
:1063B0005A208AF800000020BDE8FC9FA8462E461F
:1063C000781E01904FF0000B05E04E44C8F80060C5
:1063D000B0460BF1010B01988345F6D30020C8F8B5
:1063E0000000256065602761E760C4F808908AF8BE
:1063F00000002046E0E72DE9F04104460D46002765
:1064000001F0E8FD0746206968B1666830686060A1
:106410002069401E2061384601F0E0FD0020287010
:106420003046BDE8F081384601F0D8FD5D20287087
:106430000020F6E72DE9F04106460C4615460027F8
:106440004548007820B1112028700020BDE8F08177
:1064500001F0C0FD0746706920602068FEF7F0FC7F
:106460008046384601F0BAFD002028704046EDE72E
:106470002DE9F04105460E461446002736480078BF
:1064800018B112202070BDE8F08101F0A3FD07468D
:106490006E61384601F0A2FD0020207000BFF2E7D7
:1064A00070B504460D46002601F094FD0646D4E979
:1064B0000310884204D3304601F090FD5E2070BD89
:1064C0006068286065602069401C2061304601F0EA
:1064D00085FD0020F3E770B505460C46002601F067
:1064E00079FD06462868206068686060A868A0603A
:1064F000E868E06028692061304601F06FFDD4E96A
:106500000301401A6061002070BD70B57821134806
:10651000FEF796FF00240EE004EB44000F4901EB68
:10652000C005601C00EB400001EBC00068600CA0DF
:106530006861601C84B2042CEED304EB440007496C
:1065400001EBC0050020686005A0686108460149AC
:10655000086070BD4800002021000020B41F00200A
:106560003F0000002DE9F04106460D464FF00008BF
:106570003078022804D0012028700020BDE8F08186
:1065800001F028FD80467468E08A78B12169081D11
:1065900020610F68E08A401EE082A168206988427D
:1065A00001D1606820610020287002E01F2028705F
:1065B0000027404601F012FD3846DFE72DE9F041A3
:1065C00006460F464FF00008F748007810B100204B
:1065D000BDE8F08101F0FEFC8046F44804680068E4
:1065E00020B1F24800684068F0490860404601F078
:1065F000F5FCFCB101F0EEFC8046ED480568D5B134
:1066000000680068EA490860404601F0E7FC6E60F7
:1066100006EB8700A860EE602E61AF820020E88262
:1066200002202070002020816560E2A06061204689
:10663000FFF7C6F908E0DD4800686060DB480460E9
:10664000404601F0CBFC00242046C1E72DE9F0478D
:106650000446894615464FF0000A2078022804D0E7
:10666000012028702046BDE8F087CF48007818B197
:106670000F2028702046F6E701F0ACFC8246A07A95
:1066800010B14FF0010801E04FF00008B9F1000F20
:1066900003D0B9F1010F49D121E0B8F1000F17D1B2
:1066A000C4A060616668C24800683060C048066087
:1066B00000202070BD480068606000202081BB4839
:1066C0000460504601F08AFC00202870002705E095
:1066D000504601F083FC4920287027462DE005E054
:1066E0000223042200212046FFF7F2F8A07A0028B6
:1066F000F6D1B0A060616668AD4800683060AC4813
:10670000066000202070A948006860600020208199
:10671000A6480460504601F061FCB8F1010F01D1B8
:10672000FEF71DFC00202870002706E0504601F00F
:1067300055FC07202870274600BF00BF384692E767
:1067400070B50546002601F045FC06466C68606899
:10675000E060606820610020E082304601F03EFC8D
:10676000002070BD2DE9F0470746884615464FF0DA
:1067700000093878022804D0012028700020BDE8E4
:10678000F0878948007818B1022028700020F6E7C9
:106790008948007818B10D2028700020EFE701F03B
:1067A00019FC81467C68E08A98B12169081D206146
:1067B0000E68E08A401EE082A1682069884201D10B
:1067C00060682061484601F009FC002028703046CE
:1067D000D5E77A48006890F8340040F00400774923
:1067E000096881F8340000207449096881F835008F
:1067F00072480068C0F830803846FFF7A9F848466C
:1068000001F0ECFBFEF7ABFB01F0E4FB81466B48CB
:10681000006890F8350020B101280DD002280AD177
:1068200005E066480068466A002028700DE00026F2
:106830000E20287009E000BF394660480068FFF765
:1068400030F800260A20287000BF00BF00205B49F6
:10685000096881F834005949096881F835005749B9
:106860000968C8615549096808625449096848625D
:10687000484601F0B3FB304681E72DE9F04104467C
:106880000F4615464FF000082078022804D001205A
:1068900028700020BDE8F08101F09CFB8046A07AC2
:1068A00020B300267FB1012F0CD107E00223042280
:1068B00000212046FFF70CF8701CC6B2A07A002811
:1068C000F4D109E000BF0223042200212046FEF794
:1068D000FFFF701CC6B200BF00BF404601F07EFB48
:1068E000FEF73DFB0E2028703046D3E7404601F00E
:1068F00075FB0020287000BFCCE72DE9F04105466C
:106900000E4600272878022802D00120BDE8F08139
:1069100001F060FB0746A87A60B1002304223146EB
:106920002846FEF7D5FF384601F058FBFEF717FB67
:106930000020EBE76C68E08AA18A884204DB3846D5
:1069400001F04CFB1E20E1E7E168081DE0600E60ED
:10695000E08A401CE082D4E90210884201D16068DC
:10696000E060384601F03AFB0020CFE72DE9F04126
:1069700005460E4600272878022802D00120BDE8EF
:10698000F08101F027FB0746A87AC8B10023042252
:1069900031462846FEF79CFF384601F01FFBFEF704
:1069A000DEFA0020EBE70000210000200C000020B0
:1069B0004C0000203F000000220000203400002096
:1069C0006C68E08AA18A884204DB384601F006FB45
:1069D0001E20D4E761682069884201D1A068206147
:1069E0002069001F206120690660E08A401CE08267
:1069F000384601F0F3FA0020C1E72DE9F0410546E1
:106A00000F4616464FF000082878022802D00120D1
:106A1000BDE8F08101F0DEFA8046A87AE8B106F020
:106A2000010050B105E00023042239462846FEF754
:106A30004FFFA87A0028F6D105E00023042239464A
:106A40002846FEF745FF404601F0C8FA06F004006C
:106A500008B9FEF784FA0020DAE76C68E08AA18AB8
:106A6000884204DB404601F0B9FA1E20D0E706F068
:106A7000020058B161682069884201D1A068206194
:106A80002069001F20612069076009E0E168081D96
:106A9000E0600F60D4E90210884201D16068E060D4
:106AA000E08A401CE082404601F098FA0020AFE7FF
:106AB0002DE9F04705460C464FF0000A28780228D9
:106AC00002D00120BDE8F08701F084FA8246A87A5E
:106AD000207405F10B0804F10809002705E018F8F7
:106AE000010B09F8010B781CC7B2082FF7D36E68A9
:106AF000F08A18B130690068206001E00020206051
:106B0000F08AA080B08AE080504601F067FA002049
:106B1000D8E72DE9F04160211048FEF791FC0024F0
:106B20000DE0601C86B204EB44000C4901EBC0058B
:106B300006EB460001EBC0072F60601C84B2032CFB
:106B4000EFD304EB4400054901EBC00500202860A9
:106B5000084603490860BDE8F08100002C200020B1
:106B60004C00002070B5044600262078032801D090
:106B7000002070BD01F02EFA0646258915B1208946
:106B8000401E2081304601F029FA2846F1E770B511
:106B900005460026D748007808B1002070BD01F0F6
:106BA00019FA0646D4480468006820B1D248006843
:106BB0004068D1490860304601F010FA4CB103201A
:106BC0002070258100206060CCA060612046FEF727
:106BD000F7FE2046E2E72DE9F047044688461546D1
:106BE0004FF000092078032804D0012028702046A7
:106BF000BDE8F087BF48007818B10F202870204604
:106C0000F6E701F0E7F98146A07A08B1012700E034
:106C10000027B8F1000F03D0B8F1010F3AD119E005
:106C20008FB9B6A0606100202070B3480068606032
:106C300000202081B0480460484601F0CFF90020D0
:106C40002870002605E0484601F0C8F94920287060
:106C5000264626E005E00223012200212046FEF719
:106C600037FEA07A0028F6D1A4A060610020207031
:106C7000A14800686060002020819F480460484669
:106C800001F0ACF9012F01D1FEF769F9002028705D
:106C9000002606E0484601F0A1F9072028702646A4
:106CA00000BF00BF3046A3E72DE9F04105460E4680
:106CB000144600272878032803D001202070BDE85F
:106CC000F0818C48007810B102202070F7E78C48E2
:106CD000007810B10D202070F1E701F07BF9074634
:106CE000288940B12889401E2881384601F076F96C
:106CF00000202070E3E78348006890F8340040F0FB
:106D000001008049096881F8340000207D49096844
:106D100081F835007B48006806632846FEF718FEB8
:106D2000384601F05BF9FEF71AF901F053F907460E
:106D30007448006890F8350020B1012809D0022875
:106D400006D102E0002020700BE00E20207008E049
:106D500000BF29466B480068FEF7A3FD0A2020709B
:106D600000BF00BF00206749096881F83400654909
:106D7000096881F8350063490968C8616149096893
:106D80000862384601F02AF900BF98E72DE9F04182
:106D900004460F4615464FF000082078032804D01B
:106DA000012028700020BDE8F08101F013F9804631
:106DB000A07A20B300267FB1012F0CD107E0022377
:106DC000012200212046FEF783FD701CC6B2A07A86
:106DD0000028F4D109E000BF02230122002120464F
:106DE000FEF776FD701CC6B200BF00BF404601F042
:106DF000F5F8FEF7B4F80E2028703046D3E7404689
:106E000001F0ECF80020287000BFCCE770B5044614
:106E100000252078032801D0012070BD01F0DAF8A8
:106E20000546A07A60B10023012219462046FEF7EC
:106E30004FFD284601F0D2F8FEF791F80020ECE76C
:106E400020894FF6FF71884207D22089401C20819B
:106E5000284601F0C3F80020DFE7284601F0BEF81D
:106E60003320DAE72DE9F04704460D464FF00009DC
:106E70002078032802D00120BDE8F08701F0AAF8AD
:106E80008146A07AA87204F10B0705F102080026DA
:106E900005E017F8010B08F8010B701CC6B2082EAC
:106EA000F7D320892880484601F098F80020E3E7CE
:106EB0002DE9F04104460E461546002720780328A8
:106EC00003D001202870BDE8F08101F083F8074667
:106ED00000202870208908B1268105E0A07A08B931
:106EE000268101E049202870384601F077F800BF7C
:106EF000E9E70000210000200C0000203F00000016
:106F000022000020340000202DE9F34F85B0884690
:106F10000020019001F05EF80190FE4850F8280032
:106F200030B1019801F05AF8282007B0BDE8F08F81
:106F30000598FF2804D1F848006890F836000590BD
:106F4000F449059851F8205025B9019801F046F808
:106F50002920EAE7012D04D1019801F03FF84320F0
:106F6000E3E74FEAE80708F0070003900120B84084
:106F700000F0FF0901210398814001F0FF0A002180
:106F8000E44A059842F82010104640F8285095F839
:106F9000386095F83A00029095F839B0DF48805D86
:106FA00000EA0B00D0B1DD48805D20EA0B00DB4930
:106FB00088550846805D28B9D948007802998843E9
:106FC000D7490870D648007840EA0900D4490870CB
:106FD000D248C05D40EA0A00D049C855EC69D4B136
:106FE00004F10B00805D20EA0B0004F10B018855D1
:106FF0000846805D18B9A07A02998843A072A07AE9
:1070000040EA0900A07204F10B00C05D40EA0A00EA
:1070100004F10B01C855286A30B3286A049004981B
:1070200004681FE004F10B00805D20EA0B0004F10E
:107030000B0188550846805D18B9A07A02998843EB
:10704000A072A07A40EA0900A07204F10B00C05DB2
:1070500040EA0A0004F10B01C8550498001D049091
:1070600004980468002CDDD185F8368085F83870E6
:10707000039885F8370085F83A9085F839A001988B
:1070800000F0ACFFA7480078012801D1FDF767FFA9
:1070900000204AE72DE9FE4F06460F4690461C4663
:1070A0004FF0000900F096FF81469F48007828B114
:1070B000484600F093FF3C20BDE8FE8F954850F80D
:1070C000240060BB0120934941F82400484600F0A9
:1070D00085FF002342463946304601F002F88246D9
:1070E000002000900190034602465146029020463F
:1070F000FEF77EFC054635B98A48007801280CD198
:10710000FDF72DFF09E000F065FF81460020814971
:1071100041F82400484600F061FF2846CCE7484685
:1071200000F05CFF2820C7E702F0010343B102F042
:1071300002032BB102E0491E002308C00029FAD146
:1071400070472DE9F04F85B081468A4693461C462C
:10715000DDE90F78129D0020039000F03BFF0390C3
:107160007148007830B1039800F038FF3C2005B03A
:10717000BDE8F08F674850F8240088BB01206549BE
:1071800041F82400039800F029FF2A46414638467A
:10719000FFF7CAFF2B465A465146484600F0A1FF6A
:1071A00004901198CDE9008002953A4620460E9B46
:1071B0000499FEF71DFC064636B95A4800780128A6
:1071C0000CD1FDF7CCFE09E000F004FF0390002095
:1071D000504941F82400039800F000FF3046C6E70C
:1071E000FFE7039800F0FAFE2820C0E72DE9F04100
:1071F000054600274C48007810B14020BDE8F081DA
:107200003F2D01D13E20F9E700F0E4FE0746FF2DB7
:1072100003D14148006890F836503E4850F8254068
:1072200024B9384600F0DAFE4320E7E7012C04D108
:10723000384600F0D3FE3D20E0E714F8380F374918
:10724000085C617888432178344A505414F838092E
:107250001146085C30B994F83A10314800788843F8
:107260002F490870E06918B12046E169FEF719FB63
:10727000206A18B12046216AFDF747FEA66A16B1BA
:107280003046FEF718FD0020206384F8340084F8AF
:10729000350026480078FF2804D224480078401C96
:1072A00022490870384600F099FEFEF7F9FA00F01E
:1072B00091FE07461D48007820B11C480078401E0A
:1072C0001A490870204600F0F8FE19480078401E60
:1072D0001749087000200F4941F82500A06930B90E
:1072E00000206169886113496069086005E0D4E99C
:1072F00005014861D4E9051088610F4800686061A4
:107300000D4804600DA02065384600F067FE054872
:10731000007815E02417002034000020260000200B
:10732000250000202E000020210000202200002047
:107330002F00002040000020380000203F00000007
:10734000012801D1FDF70BFE002057E72DE9F041A0
:10735000044600273F2C02D13E20BDE8F081FF2CDF
:107360000BD100F037FE0746F948006890F83B6003
:10737000384600F033FE3046EFE700F02BFE0746BC
:10738000F44850F8245025B9384600F027FE432031
:10739000E3E7012D04D1384600F020FE3D20DCE774
:1073A0003F2085F83B00384600F018FE0020D4E767
:1073B0002DE9F04706460F4614464FF00008E64810
:1073C000007820B1112020700020BDE8F08700F087
:1073D00001FE8046FF2E03D1DD48006890F836603C
:1073E000DC4850F8265035B9404600F0F7FD432000
:1073F00020700020E9E7012D06D1404600F0EEFDA7
:10740000432020700020E0E7286D38603868FDF7E1
:1074100017FD8146404600F0E1FD002020704846FF
:10742000D3E72DE9F04106460F4614464FF0000819
:10743000C948007818B112202070BDE8F08100F032
:10744000C9FD8046FF2E03D1C148006890F8366020
:10745000C04850F826502DB9404600F0BFFD4320EB
:107460002070EAE7012D05D1404600F0B7FD43202A
:107470002070E2E72F65404600F0B0FD002020704C
:1074800000BFDAE770B50546002600F0A3FD06460A
:10749000B04850F8254024B9304600F09FFD462002
:1074A00070BD012C04D1304600F098FD4320F7E771
:1074B00094F8340000F0080060B314F8340F00F0C2
:1074C000F700207014F83409F8B9206BC8B93834C3
:1074D000A078A24909780843A04908702078A049FB
:1074E000085C6178084314F838199D4A50543046B6
:1074F00000F074FD9B480078012809D1FDF72FFDAD
:1075000006E0304600F06AFD02E0304600F066FD1D
:107510000020C5E7304600F061FD4420C0E72DE9BA
:10752000F04707460D464FF0000A002028606860CB
:1075300000F050FD8246FF2F03D18548006890F887
:107540003670844850F827402CB9504600F046FD6C
:107550004320BDE8F087012C04D1504600F03EFDE9
:107560004320F6E7207C00F0010020B9504600F0EF
:1075700035FD4520EDE70026D4F80C90D4F80880BE
:10758000504600F02BFD00E0761C58F8041B002943
:10759000FAD02E60A9EB060068600020D9E72DE93B
:1075A000F04105464FF0000800F014FD8046FF2D25
:1075B00005D16748006890F83650012608E0644815
:1075C000006890F83600A84201D1012600E00026AC
:1075D000604850F825402CB9404600F0FFFC482098
:1075E000BDE8F081012C04D1404600F0F7FC4320B7
:1075F000F6E794F838705A48C05D94F8391088431B
:107600005749C8550846C05D30B994F83A105348F8
:10761000007888435149087094F8340040F008001D
:1076200084F83400404600F0D9FC012E01D1FDF76A
:1076300096FC0020D4E72DE9F04105460E460027D0
:1076400000F0C8FC0746FF2D03D14148006890F8C0
:107650003650404850F825402CB9384600F0BEFC62
:107660002920BDE8F081012C04D1384600F0B6FC99
:107670004320F6E7582221463046FEF7AFF9384658
:1076800000F0ACFC0020ECE72DE9F04704460E4684
:1076900017464FF0000900F09DFC8146FF2C02D1F7
:1076A0002B48056802E02B4850F8245005F154009F
:1076B00050F82680484600F091FC00203870404683
:1076C000BDE8F08770B50446002600F083FC06464E
:1076D0002548007830B196202070304600F07EFCBE
:1076E000012070BD204805780078401C1E490870B4
:1076F000304600F073FC002020702846F1E72DE9A9
:10770000F04704460E46174698464FF0000900F031
:1077100061FC8146FF2C02D10D48056802E00D484E
:1077200050F8245005F1540040F82670484600F007
:1077300055FC002088F80000BDE8F08710B504482B
:10774000006800F0C4FCFF20FFF750FD10BD0000F2
:1077500034000020241700202100002025000020F4
:10776000260000202E0000205000002070B50546A5
:1077700000266348007800B170BD6248007800B10F
:10778000FAE71DB300F026FC06465F48006890F853
:1077900038405E48005D5C49096891F839108843BB
:1077A0005A4908550846005D40B95748006890F8A6
:1077B0003A10574800788843554908705248006885
:1077C0000563304600F00AFCFDF7C9FB00BFD3E7B4
:1077D0002DE9F04105460E4617461C4648480078FC
:1077E00010B15520BDE8F0814648007808B132203C
:1077F000F8E74FF47A7060434FF47A71B0FBF1F11F
:107800004FF461606843C6EB061200EB8200384417
:1078100000EB4002C2EBC01001EBC0084046FFF78E
:10782000A5FF0020DEE770B5054600263F2D01D3F9
:107830002A2070BD00F0CEFB0646364850F82540A1
:1078400024B9304600F0CAFB4320F2E7012C04D1F2
:10785000304600F0C3FB4320EBE7206B20B93046F5
:1078600000F0BCFB5020E4E70020206394F83400D3
:1078700000F0370040B114F8340F20F037002070CA
:1078800001206070343C02E0002084F8350094F858
:10789000340000F00800A8B93834A0781C490978F1
:1078A00008431B49087020781849085C6178084330
:1078B00014F83819154A5054304600F08FFBFDF784
:1078C0004EFB02E0304600F089FB0020B1E770B5C6
:1078D000002500F07FFB05460F480468284600F0AD
:1078E0007DFB204670BD70B50446002500F072FB9C
:1078F000054609480460284600F070FB70BD000092
:10790000210000202200002034000020260000205A
:10791000250000202417002054000020F8480068AB
:1079200008B900207047F6480168F54AC868106039
:107930000020C8600861F3480088401CF14A1080AC
:10794000F1480088401EF04A10800846EAE72DE919
:10795000F05F06460F4690469946DDE90ABA0C9D4F
:10796000EA48007820B18B2028700020BDE8F09F05
:10797000FDF766FEFFF7D2FF04462CB9FDF7C4FE03
:10798000862028700020F1E7012084F82500A661F8
:10799000E76184F82480C4F80490C4F808B0BAF110
:1079A000000F02D1DAA0206201E0C4F820A0FDF7A8
:1079B000ABFE002028702046D8E7002180F8251073
:1079C00080F82410C161416141608160D0A10162F1
:1079D00000210161CA490968C160C9490860C949F3
:1079E0000988491EC74A1180C7490988491CC64AE7
:1079F0001180704730B5057D05F00704C54D05EBD6
:107A0000C4031D68854205D1C168196039B10025DC
:107A10000D6104E00169C268CA6002B1116101250B
:107A200080F825500025C56005619D886D1E9D80EC
:107A300030BD70B505460C462878642803D08920EF
:107A40002070002070BDB148007818B18B202070E4
:107A50000020F7E7FDF7F4FD95F82500D8B10128DF
:107A60000FD002280ED003281BD12846FFF7C2FFF3
:107A70002846FFF7A2FFFDF747FE002020700120F7
:107A8000E0E700BF2846FFF798FFFDF73DFE002026
:107A900020700120D6E7FDF737FE872020700020F8
:107AA000D0E7FDF731FE8D2020700020CAE72DE9D8
:107AB000F04105460E4614462878642804D08920F3
:107AC00020700020BDE8F0819048007818B11120A6
:107AD00020700020F6E7FDF7B3FD95F8250098B17A
:107AE000012804D0022803D0032813D100BF00BF0F
:107AF000286A30603068FDF7A3F90746FDF704FEF9
:107B0000002020703846DDE7FDF7FEFD872020705D
:107B10000020D7E7FDF7F8FD8D2020700020D1E789
:107B200070B504460D462078642803D0892028705B
:107B3000002070BD7548007818B18B202870002097
:107B4000F7E7FDF77DFD94F8250070B301280DD00F
:107B5000022825D003282FD16F4960690968461A89
:107B6000FDF7D2FD002028703046E2E794F82400AB
:107B700001280CD0022809D1A06908B9E66900E003
:107B8000A669FDF7C1FD0020287006E000BFA669C8
:107B9000FDF7BAFD0020287000BF00BF3046C8E7DF
:107BA000FDF7B2FD00202870C3E7FFE7FDF7ACFD4D
:107BB000872028700020BCE7FDF7A6FD8D202870E7
:107BC0000020B6E770B505460C462878642803D037
:107BD00089202070002070BD4C48007818B18B209F
:107BE00020700020F7E7FDF72BFD95F8256036B1F2
:107BF000012E05D0022E04D0032E06D102E000BFD4
:107C000000BF00BF0020207002E08D20207000BF68
:107C100000BFFDF779FD3046DDE770B50B46032563
:107C200080F82550012B05D13B4EC5693668354497
:107C300045610CE085692DB9374EC5693668354414
:107C4000456104E0344E8569366835444561057DFB
:107C500005F007042F4D05EBC4010D682DB9086030
:107C60000025C56001258D8006E00A680860C260B5
:107C700010618D886D1C8D800025056170BD70B50B
:107C800005460C462878642803D0892020700020FF
:107C900070BD1E48007818B18B2020700020F7E7D7
:107CA000FDF7CEFC95F82500E8B1012810D0022898
:107CB0000FD003281DD12846FFF79CFE002128463F
:107CC000FFF7ABFFFDF720FD002020700120DFE76C
:107CD00000BF00212846FFF7A0FFFDF715FD00209B
:107CE00020700120D4E7FDF70FFD872020700020D1
:107CF000CEE7FDF709FD8D2020700020C8E70000C9
:107D0000680000205A0000205800002021000020B8
:107D10003F0000000C2500205C0000202DE9F04110
:107D200005460F4690461C462878642804D08920D2
:107D300020700020BDE8F0817D48007818B18B20CC
:107D400020700020F6E7FDF77BFC95F82500002861
:107D500032D001282AD0022827D0032832D1284641
:107D6000FFF748FE00202070B7B1032F02D0042F88
:107D700013D108E06E681EB12846A968B04701E03B
:107D80008F2020700CE06E681EB141462846B04737
:107D900001E08F20207003E002E08420207000BF0B
:107DA00000BFFDF7B1FC0120C4E700BFFDF7ACFC4C
:107DB0008E2020700120BDE7FDF7A6FC87202070F3
:107DC0000020B7E7FDF7A0FC8D2020700020B1E770
:107DD00010B558480068FFF719F80446204610BD52
:107DE00008B500BF00BF6A46002152480068FEF790
:107DF0005BFFFDF725FC50480068401C4E490860B9
:107E00000846007800F007084C4800EBC8073C68BB
:107E10001AE0E668484960690968884213D120463B
:107E2000FFF7E8FD94F82400022804D10121204640
:107E3000FFF7F3FE02E0022084F82500656815B123
:107E40002046A168A8473446002CE2D1FDF75CFC2F
:107E5000C9E700B587B0032000218022384BCDE967
:107E60000132CDE903104FF6FD703D23354A0090F5
:107E70003548FFF766F906AA34A13D20FFF7D1FA8D
:107E800007B000BDF8B54FF420713448FDF7D8FABB
:107E900040212A48FDF7D4FA002515E0681C86B277
:107EA00005EB85002D4901EBC00406EB860001EBD4
:107EB000C00764202070002084F82500E760AFF23E
:107EC000B0102062681C85B20F2DE7D305EB85004A
:107ED000224901EBC00464202070002084F82500B2
:107EE000E060AFF2D41020620020134908601C4902
:107EF000088010201B49088018481B490860012091
:107F0000FEF745FE194908600020FEF740FE0949CA
:107F100008606A4616A115480068FCF7CCFF6A465F
:107F200018A104480068FCF7C6FFFFF792FFF8BDF0
:107F300021000020640000205C0000200C250020AF
:107F40000C23002008250020E17D000075432F4F01
:107F5000532D494920546D72000000008C200020F0
:107F60005A00002058000020680000206000002017
:107F700075432F4F532D494920546D724C6F636BDD
:107F80000000000075432F4F532D494920546D7256
:107F90005369676E616C00007047704770477047A7
:107FA0007047704770477047EFF3098141B1F1EEB8
:107FB000101A40F8041D20ED200A29490A681060B3
:107FC0007047B0EC200A02C8E1EE101A25490A6891
:107FD00010607047EFF3108072B6704780F310881E
:107FE000704721484FF0FF010170002080F309889D
:107FF0001E48016881F308881D48012101701D4851
:108000004FF08051016062B6FEE71A484FF0805190
:108010000160704717484FF080510160704772B699
:10802000EFF3098028B1203880E8F00F0C49096887
:10803000086000B5104880475DF804EB0F48104910
:108040000A780270064807490A680260106890E8DA
:10805000F00F203080F309884EF0F40E62B67047BE
:10806000340000203C00002022ED00E06C000020E5
:108070002E00002004ED00E09F820000230000207D
:1080800024000020A648802102E0491E002204C0EE
:108090000029FAD1A34AA44B1A601A46126822F0AA
:1080A00007021A600022A14B1A807047704710B572
:1080B00004462046FFF770FF10BD10B50446204669
:1080C000FFF76BFF10BD10B5FFF768FF10BD10B5CF
:1080D00004462046FFF764FF10BD10B5FFF75FFFB1
:1080E00010BD70B50446101D20F007004FF08076DB
:1080F000051F28462E60051F28462C608C4E051F44
:1081000028462E604FF01236051F28462E604FF08D
:108110000336051F28462E604FF00236051F2846FD
:108120002E607610051F28462E60051F2846296000
:108130004FF01136051F28462E604FF01036051FF0
:1081400028462E604FF00936051F28462E604FF056
:108150000836051F28462E604FF00736051F2846B3
:108160002E604FF00636051F28462E604FF005366C
:10817000051F28462E604FF00436051F28462E6046
:1081800003F00405002D7DD0F605051F28462E605E
:10819000684E051F28462E60674E051F28462E6034
:1081A000664E051F28462E60654E051F28462E6028
:1081B000644E051F28462E60634E051F28462E601C
:1081C000624E051F28462E60614E051F28462E6010
:1081D000604E051F28462E605F4E051F28462E6004
:1081E0005E4E051F28462E605D4E051F28462E60F8
:1081F0005C4E051F28462E605B4E051F28462E60EC
:108200005A4E051F28462E604FF08346051F28460C
:108210002E60574E051F28462E60564E051F2846D5
:108220002E60554E051F28462E60544E051F2846C9
:108230002E60534E051F28462E60524E051F2846BD
:108240002E60514E051F28462E604FF08246051FB6
:1082500028462E604D4E051F28462E604C4E051FA9
:1082600028462E604B4E051F28462E604FF0814653
:10827000051F28462E60484E051F28462E603602F0
:10828000051F00E00AE028462E604FF07E56051FCD
:1082900028462E600026051F28462E6070BD10B5AA
:1082A000FFF77FFE10BD10B504462046FFF77AFEAB
:1082B00010BD10B5FFF777FE1C480088401C1B4915
:1082C00008800846008818B100200880FFF780FD6C
:1082D00010BD10B5FFF77EFE044630480078401C04
:1082E0002E4908702046FFF779FEFDF76DFAFDF77D
:1082F0006FF910BD01464A1E4FF0E0235A61284A2B
:10830000106820F07F4000BF10601A46126942F0EA
:1083100005021A611A46126942F002021A61704798
:108320004C2500204C2700206C000020700000200D
:108330003D7700000000F8410000F0410000E841F6
:108340000000E0410000D8410000D0410000C841D9
:108350000000C0410000B8410000B0410000A84149
:108360000000A041000098410000904100008841B9
:108370000000704100006041000050410000404199
:108380000000304100002041000010410000E040AA
:108390000000C0400000A04000004040210000203C
:1083A00020ED00E01D481E481E481F481F48204879
:1083B000204821482148224822482348234824486D
:1083C000244825482548264826482748274828483D
:1083D0002848294829482A482A482B482B482C480D
:1083E0002C482D482D482E482E482F482F483048DD
:1083F00030483148314832483248334833483448AD
:10840000344835483548364836483748374838487C
:1084100038483948394800BF70470000C8AD0000EF
:10842000CCAD0000D2AD0000D4AD0000D0AD000056
:10843000D6AD0000D8AD0000DAAD0000DCAD000024
:10844000DEAD0000E0AD0000E2AD0000E4AD0000F4
:10845000E6AD0000E8AD0000EAAD0000ECAD0000C4
:10846000EEAD0000F0AD0000F2AD0000F4AD000094
:10847000F6AD0000F8AD0000FAAD0000FCAD000064
:10848000FEAD000000AE000002AE000004AE000031
:1084900006AE000008AE00000AAE00000CAE000000
:1084A0000EAE000010AE000012AE000014AE0000D0
:1084B00016AE000018AE00001AAE00001EAE00009E
:1084C00020AE000022AE000024AE00008C20002070
:1084D0000C25002028AE00002AAE00002CAE0000C3
:1084E0002EAE000030AE000032AE000034AE000010
:1084F00036AE000038AE000026AE00003AAE0000F6
:10850000DFF83000016841F470010160BFF34F8F64
:10851000DFF82400016821F040410160BFF36F8F54
:1085200006480047FEE7FEE7FEE7FEE7FEE7FEE758
:10853000FEE7000088ED00E034EF00E001020000FB
:1085400070470B490860704709480068704710B5CC
:10855000044622460221074800F0D9F80CB9012050
:1085600000E0002002460121024800F0D0F810BDD2
:1085700074000020007000402DE9F04104460E46D2
:1085800015461F46B4F1402F02D07548844203D1EE
:108590007448F8F7F7FE98E07348844202D07348B5
:1085A000844204D16F48401CF8F7ECFE8DE070481F
:1085B000844202D06F48844204D16A48801CF8F794
:1085C000E1FE82E06C48844202D06C48844204D1CF
:1085D0006448C01CF8F7D6FE77E06948844202D0B0
:1085E0006848844204D15F48001DF8F7CBFE6CE078
:1085F0006548844202D06548844204D15948401DF0
:10860000F8F7C0FE61E06248844202D061488442CB
:1086100004D15448C01DF8F7B5FE56E05E488442C8
:1086200002D05E48844204D14E480830F8F7AAFED2
:108630004BE05B48844204D14A480930F8F7A2FE77
:1086400043E05848844204D146480A30F8F79AFE7D
:108650003BE05548844204D142480B30F8F792FE83
:1086600033E05248844204D13E480C30F8F78AFE89
:108670002BE04F48844204D13A480D30F8F782FE8F
:1086800023E04C48844204D136480E30F8F77AFE95
:108690001BE04948844204D132480F30F8F772FE9B
:1086A00013E04648844204D12E481030F8F76AFEA1
:1086B0000BE04348844204D12A481130F8F762FEA7
:1086C00003E04FF0FF30BDE8F0812DB92A46314676
:1086D0002046F7F7D3FD18E0012D0BD12A4631468D
:1086E0002046F7F7CBFD3B46012231462046F7F7FF
:1086F00052FE0AE0022D05D12A4631462046F7F700
:10870000BDFD02E04FF0FF30DDE70020DBE770B594
:1087100005460C4616462A48854201D8802C02DDC3
:108720004FF0FF3070BD012E05D12246214628466C
:10873000F7F7CBFF05E0E043C2B221462846F7F742
:10874000C4FF0020EEE770B505460C4621462846DA
:10875000F7F7B5FFA04201D1012070BD0020FCE772
:1087600000800540000800F00050004000900540E7
:108770000060004000A005400070004000B00540CF
:108780000040024000C005400050024000D00540BB
:108790000070024000F0054000D003400000064099
:1087A0000010064000200640003006400040064011
:1087B0000050064000600640007006400080064001
:1087C000009006402DE9F04105460C4616461F462E
:1087D000002E69D115B1012D63D130E0F748F8F7CB
:1087E000D1FDF748F8F7CEFDF648F8F7FFF8F64860
:1087F000F8F7FCF80421F548F8F72FF80821F348BA
:10880000F8F71CF8F248844208D1FFF79DFE804635
:1088100001224146EF48F8F754F90FE0EE48844250
:1088200008D1FFF791FE804600224146E948F8F75B
:1088300048F903E04FF0FF30BDE8F08131E0DF4858
:10884000401CF8F79FFDDE48401DF8F79BFDE3480C
:10885000F8F7CCF8E248F8F7C9F80121E148F7F752
:10886000FCFF0221DF48F7F7E9FFD948844208D12D
:10887000FFF76AFE804601224146DB48F8F721F9FE
:108880000EE0D548844208D1FFF75EFE8046002204
:108890004146D548F8F715F902E04FF0FF30CBE735
:1088A00000BF00BF0020C7E7012E3AD115B1012D4E
:1088B00034D118E0C148F8F765FDC148F8F762FD0A
:1088C000C048F8F793F8C048F8F790F80421BF487B
:1088D000F7F7C3FF0821BD48F7F7B0FF3946BD4899
:1088E000F8F71EF91AE0B548401CF8F74BFDB448FC
:1088F000401DF8F747FDB948F8F778F8B848F8F799
:1089000075F80121B748F7F7A8FF0221B548F7F736
:1089100095FF3946B448F8F703F900BF00BF0020BF
:108920008AE74FF0FF3087E72DE9F0470746884692
:1089300016461D464FF00009FFF74CFB814635B93E
:108940004846FFF74BFB4FF0FF30BDE8F087002FA4
:108950006AD100BF9F48F8F78BF90028FAD10022AE
:1089600041469C48F8F77DF9012D1BD13178994893
:10897000F8F7A1F907219748F8F78CF99548F8F727
:108980008BF920B14846FFF729FBA81EDDE700BFA1
:108990009048F8F76DF90028FAD14846FFF71EFB1A
:1089A0000020D2E700243CE044B9315D8948F8F763
:1089B00082F903218748F8F76DF913E0681EA04299
:1089C00008D1315D8348F8F776F905218148F8F739
:1089D00061F907E0315D7F48F8F76DF901217D48C5
:1089E000F8F758F97B48F8F757F998B1681EA04294
:1089F0000AD07848F8F750F900F01000102803D09A
:108A000004217448F8F746F94846FFF7E7FA4FF0B3
:108A1000FF309AE700BF6F48F8F72AF90028FAD12B
:108A2000641CAC42C0D37DE0012F75D100BF6E48FD
:108A3000F8F71EF90028FAD1002241466A48F8F7F3
:108A400010F9012D1BD131786748F8F734F9072167
:108A50006548F8F71FF96448F8F71EF920B1484651
:108A6000FFF7BCFAA81E70E700BF5F48F8F700F9EF
:108A70000028FAD14846FFF7B1FA002065E7002444
:108A800046E044B9315D5848F8F715F903215648D6
:108A9000F8F700F913E0681EA04208D1315D524892
:108AA000F8F709F905215048F8F7F4F807E0315DC7
:108AB0004D48F8F700F901214B48F8F7EBF84A4820
:108AC000F8F7EAF828B14846FFF788FA4FF0FF3088
:108AD0003BE74548F8F7E0F898B1681EA0420AD095
:108AE0004148F8F7D9F800F01000102803D004210D
:108AF0003D48F8F7CFF84846FFF770FA4FF0FF30DF
:108B000023E700BF3848F8F7B3F80028FAD1641C0F
:108B1000AC42B6D306E0FFE74846FFF75FFA4FF0F6
:108B2000FF3012E74846FFF759FA00200DE72DE91C
:108B3000F0470746884616461D464FF00009FFF7E6
:108B400049FA814635B94846FFF748FA4FF0FF30F9
:108B5000BDE8F087002F7CD100BF1E48F8F788F8E9
:108B60000028FAD1012241461A48F8F77AF8012D77
:108B70001BD107211748F8F78DF81648F8F78CF83D
:108B800020B14846FFF72AFAA81EE1E700BF1148C6
:108B9000F8F76EF80028FAD10E48F8F78EF8307022
:108BA0004846FFF71BFA0020D2E700244DE0ECB95D
:108BB0000B210848F8F76EF824E00000002000F0D0
:108BC000010800F002080100020C01000050004002
:108BD000801A060000000240A08601000200060084
:108BE000020406000060024000100240681EA0421D
:108BF00004D105215248F8F74DF803E00921504807
:108C0000F8F748F84E48F8F747F898B1681EA042C0
:108C10000AD04B48F8F740F800F01000102803D0B5
:108C200004214748F8F736F84846FFF7D7F94FF0E0
:108C3000FF308DE700BF4248F8F71AF80028FAD154
:108C40003F48F8F73AF83055641CAC42AFD36BE0BC
:108C5000FFE7012F62D100BF3A48F8F709F8002872
:108C6000FAD1012241463748F7F7FBFF012D1BD10E
:108C700007213448F8F70EF83248F8F70DF820B11C
:108C80004846FFF7ABF9A81E62E700BF2D48F7F78B
:108C9000EFFF0028FAD12B48F8F70FF8307048465C
:108CA000FFF79CF9002053E7002434E024B90B219E
:108CB0002448F7F7EFFF0BE0681EA04204D105211E
:108CC0002048F7F7E7FF03E009211E48F7F7E2FF26
:108CD0001C48F7F7E1FF98B1681EA0420AD0194876
:108CE000F7F7DAFF00F01000102803D00421154830
:108CF000F7F7D0FF4846FFF771F94FF0FF3027E74D
:108D000000BF1048F7F7B4FF0028FAD10D48F7F775
:108D1000D4FF3055641CAC42C8D305E04846FFF789
:108D20005DF94FF0FF3013E74846FFF757F9002091
:108D30000EE70346002070470346002070470000FE
:108D4000000002400010024010B50121FA48F9F776
:108D50004CF904462146F848F9F74DF9FCF722FC96
:108D60000EE0F548F9F7E9F8F449F54A1268885435
:108D7000F3480068401CF249086008460078086023
:108D8000ED48F9F7CEF80028EBD1FCF721FC10BD37
:108D900010B50121EB48F9F728F904462146E948C6
:108DA000F9F729F9FCF7FEFB0EE0E648F9F7C5F8FC
:108DB000E549E64A12688854E4480068401CE349E3
:108DC0000860084600780860DE48F9F7AAF800282D
:108DD000EBD1FCF7FDFB10BD10B50121DC48F9F724
:108DE00004F904462146DA48F9F705F9FCF7DAFBFD
:108DF0000EE0D748F9F7A1F8D649D74A1268885447
:108E0000D5480068401CD4490860084600780860CE
:108E1000CF48F9F786F80028EBD1FCF7D9FB10BD55
:108E200010B50121CD48F9F7E0F804462146CB48BA
:108E3000F9F7E1F8FCF7B6FB0EE0C848F9F77DF862
:108E4000C749C84A12688854C6480068401CC549CA
:108E50000860084600780860C048F9F762F8002802
:108E6000EBD1FCF7B5FB10BD10B50121BE48F9F7F9
:108E7000BCF804462146BC48F9F7BDF8FCF792FB64
:108E80000EE0B948F9F759F8B849B94A1268885458
:108E9000B7480068401CB64908600846007808607A
:108EA000B148F9F73EF80028EBD1FCF791FB10BD73
:108EB00010B50121AF48F9F798F804462146AD48AE
:108EC000F9F799F8FCF76EFB0EE0AA48F9F735F8C8
:108ED000A949AA4A12688854A8480068401CA749B2
:108EE0000860084600780860A248F9F71AF80028D8
:108EF000EBD1FCF76DFB10BD10B50121A048F9F7CF
:108F000074F8044621469E48F9F775F8FCF74AFBC9
:108F10000EE09B48F9F711F89A499B4A1268885469
:108F200099480068401C9849086008460078086025
:108F30009348F8F7F6FF0028EBD1FCF749FB10BD8A
:108F400010B501219148F9F750F8044621468F48A1
:108F5000F9F751F8FCF726FB0EE08C48F8F7EDFF27
:108F60008B498C4A126888548A480068401C894999
:108F700008600846007808608448F8F7D2FF0028A7
:108F8000EBD1FCF725FB10BD2DE9F04704468846E0
:108F900015461E46089F84BB7F48F8F7F3F97F48C3
:108FA000F8F7F0F90120F7F721FD40F20140F7F75B
:108FB0001DFD03214FF04020F7F7C7FCFFF7C4FA6F
:108FC000814645EA060040EA0703424649466F48A3
:108FD000F8F714FF72490520FBF7D1FB0520FBF7DA
:108FE000C4FB1520F7F79CFF60211520F7F776FFEB
:108FF00050216648F8F7F1FFB0E1FFE7012C31D1CD
:109000006548401CF8F7BEF96448401CF8F7BAF907
:109010004FF00110F7F7EAFC6248F7F7E7FC03218D
:109020006148F7F792FCFFF78FFA814645EA0600A0
:1090300040EA0703424649465148F8F7DFFE5B49DC
:109040000620FBF79CFB0620FBF78FFB1620F7F7AB
:1090500067FF60211620F7F741FF50214848F8F7D5
:10906000BCFF7BE1022C32D14B48801CF8F78AF917
:109070004A48F8F787F941F60100F7F7B7FC41F6DF
:109080000140F7F7B3FCC0214FF04020F7F75DFC3B
:10909000FFF75AFA814645EA060040EA07034246CE
:1090A00049463448F8F7AAFE41492120FBF767FBFF
:1090B0002120FBF75AFB3120F7F732FF60213120E6
:1090C000F7F70CFF50212B48F8F787FF46E1032CF8
:1090D00073D13148C01CF8F755F93048F8F752F908
:1090E00041F20100F7F782FC41F20140F7F77EFC04
:1090F00030214FF04020F7F728FCFFF725FA814692
:1091000045EA060040EA0703424649461648F8F792
:1091100075FE28493820FBF732FB3820FBF725FB8A
:109120004820F7F7FDFE60214820F7F7D7FE5021D1
:109130000D48F8F752FF11E1003001404C2E00209D
:10914000B0000020002001404C2D0020A80000208D
:10915000001001404C2C0020A00000200000014025
:109160004C2B00209800002000F000404C2A0020EA
:109170009000002000E000404C29002088000020E2
:1091800000D000404C2800208000002000C000409B
:109190004C27002078000020001800F0000800F0A4
:1091A000418F00000104010000500040F98E0000D2
:1091B000B18E0000698E0000FFE7042C31D1F64823
:1091C000F8F7E0F8F548F8F7DDF840F60100F7F7B2
:1091D0000DFC40F60140F7F709FC0C214FF0402050
:1091E000F7F7B3FBFFF7B0F9814645EA060040EA1E
:1091F000070342464946EA48F8F700FEE9493920A4
:10920000FBF7BDFA3920FBF7B0FA4920F7F788FEE3
:1092100060214920F7F762FE5021E148F8F7DDFEB2
:109220009CE0052C30D1DC48401CF8F7ABF8DB485B
:10923000801CF8F7A7F8DC48F7F7D8FBDB48F7F70E
:10924000D5FBC021DA48F7F780FBFFF77DF98146AF
:1092500045EA060040EA070342464946D548F8F782
:10926000CDFDD5493A20FBF78AFA3A20FBF77DFA83
:109270004A20F7F755FE60214A20F7F72FFE5021CC
:10928000CC48F8F7AAFE69E0062C30D1C248801C11
:10929000F8F778F8C1480D30F8F774F8C748F7F7D1
:1092A000A5FBC748F7F7A2FB0321C648F7F74DFB1C
:1092B000FFF74AF9814645EA060040EA07034246BD
:1092C0004946C148F8F79AFDC0493B20FBF757FAD9
:1092D0003B20FBF74AFA4B20F7F722FE60214B2098
:1092E000F7F7FCFD5021B848F8F777FE36E0072C79
:1092F00030D1A948C01CF8F745F8A848801CF8F7F9
:1093000041F8B348F7F772FBB248F7F76FFB30212B
:10931000A748F7F71AFBFFF717F9814645EA060059
:1093200040EA070342464946AB48F8F767FDAB49B8
:109330003C20FBF724FA3C20FBF717FA4C20F7F708
:10934000EFFD60214C20F7F7C9FD5021A248F8F746
:1093500044FE03E04FF0FF30BDE8F0870020FBE75C
:109360002DE9F04105460E4617460024A046FEF7BB
:1093700031FE804675B904E0315D9948F8F7FAFD91
:10938000641CBC42F8D300BF9548F8F705FE0028DE
:10939000FAD17DE0012D0ED104E0315D9148F8F75E
:1093A000E9FD641CBC42F8D300BF8E48F8F7F4FD19
:1093B0000028FAD16CE0022D0ED104E0315D8A481C
:1093C000F8F7D8FD641CBC42F8D300BF8648F8F714
:1093D000E3FD0028FAD15BE0032D0ED104E0315DFE
:1093E0008248F8F7C7FD641CBC42F8D300BF7F4831
:1093F000F8F7D2FD0028FAD14AE0042D0ED104E09E
:10940000315D6748F8F7B6FD641CBC42F8D300BF75
:109410006348F8F7C1FD0028FAD139E0052D0ED1D7
:1094200004E0315D6348F8F7A5FD641CBC42F8D345
:1094300000BF6048F8F7B0FD0028FAD128E0062DFB
:109440000ED104E0315D6048F8F794FD641CBC4225
:10945000F8D300BF5C48F8F79FFD0028FAD117E069
:10946000072D0ED104E0315D5B48F8F783FD641CE5
:10947000BC42F8D300BF5848F8F78EFD0028FAD157
:1094800006E04046FEF7AAFD4FF0FF30BDE8F08150
:109490004046FEF7A3FD0020F8E72DE9F04107461E
:1094A0000D4616460024A046FEF794FD8046082F80
:1094B00071D2DFE807F0041F3A55B5D0EBF4002471
:1094C00014E04B4800684B490968884200D10FE01E
:1094D000494847490968405C285545480068401C90
:1094E00043490860084600780860641CB442E8D329
:1094F00000BF03E1002414E04048006840490968C7
:10950000884200D10FE03F483C490968405C28553B
:109510003A480068401C39490860084600780860ED
:10952000641CB442E8D300BFE8E0002414E03648ED
:10953000006836490968884200D10FE03448324952
:109540000968405C285530480068401C2E49086076
:10955000084600780860641CB442E8D300BFCDE040
:10956000002414E02B4800682B490968884200D188
:109570000FE02A4827490968405C285525480068BB
:10958000401C24490860084600780860641CB44206
:10959000E8D300BFB2E0B0E0041800F0000800F02B
:1095A00000000140218E000001180200011C020091
:1095B0000060004000100140D98D000001000D0046
:1095C00001040D000050064000200140918D000074
:1095D000011002000114020000300140498D00001A
:1095E00000C0004000D0004000E0004000F000401B
:1095F0007C000020780000204C2700208400002000
:10960000800000204C2800208C00002088000020D2
:109610004C29002094000020900000204C2A0020BB
:10962000002414E03948006839490968884200D1AB
:109630000FE0384835490968405C285533480068D0
:10964000401C32490860084600780860641CB44237
:10965000E8D300BF52E0002414E02F4800682F49EF
:109660000968884200D10FE02D482B490968405C09
:10967000285529480068401C27490860084600789A
:109680000860641CB442E8D300BF37E0002415E052
:109690002448006824490968884201D110E011E09B
:1096A000224820490968405C28551E480068401C33
:1096B0001C490860084600780860641CB442E7D37F
:1096C00000BF1BE0002414E019480068194909682C
:1096D000884200D10FE0184815490968405C2855B8
:1096E00013480068401C124908600846007808606A
:1096F000641CB442E8D300BF00E000BF00BF404696
:10970000FEF76CFC2046BDE8F08100009C000020C4
:10971000980000204C2B0020A4000020A000002076
:109720004C2C0020AC000020A80000204C2D002074
:10973000B4000020B00000204C2E002010B50549D8
:10974000012000F081F84FF4E131012000F069FBC5
:1097500010BD0000801A060038B520208DF80000EA
:109760005E208DF8010002236A466821FE480078D9
:10977000FFF7DAF80446002C02DA4FF0FF3038BD6C
:1097800021208DF80000C7208DF8010002236A46D1
:109790006821F5480078FFF7C7F80446002C02DA84
:1097A0004FF0FF30EBE722208DF8000001208DF80C
:1097B000010002236A466821EB480078FFF7B4F8FD
:1097C0000446002C02DA4FF0FF30D8E707208DF86E
:1097D000000040208DF8010002236A466821E2481B
:1097E0000078FFF7A1F80446002C02DA4FF0FF30B2
:1097F000C5E70020C3E738B508208DF80000202019
:109800008DF8010002236A466821D7480078FFF7E7
:109810008BF80446002C02DA4FF0FF3038BD0920E7
:109820008DF8000045208DF8010002236A4668216A
:10983000CD480078FFF778F80446002C02DA4FF0A4
:10984000FF30EBE70020E9E770B505460E46C64855
:10985000057000231A4631460078FEF7B3FF044630
:10986000002C02DA4FF0FF3070BDFFF7C4FF044652
:10987000002C02DA4FF0FF30F6E7FFF76DFF0446E9
:10988000002C02DA4FF0FF30EEE70020ECE77CB569
:1098900004460620019000200090012301AA6821BF
:1098A000B1480078FFF740F80546002D02DA4FF086
:1098B000FF307CBD01236A466821AB480078FFF782
:1098C00036F90546002D02DA4FF0FF30F1E79DF83A
:1098D000000000F00F009DF80010090901EB810164
:1098E00000EB410020700020E3E77CB50446052032
:1098F000019000200090012301AA68219A48007875
:10990000FFF712F80546002D02DA4FF0FF307CBD5C
:1099100001236A46682194480078FFF708F9054654
:10992000002D02DA4FF0FF30F1E79DF8000000F063
:109930000F009DF80010C1F3001101EB810100EB55
:10994000410020700020E2E77CB50446042001902D
:1099500000200090012301AA682183480078FEF7C7
:10996000E3FF0546002D02DA4FF0FF307CBD0123F6
:109970006A4668217C480078FFF7D9F80546002D33
:1099800002DA4FF0FF30F1E79DF8000000F00F0021
:109990009DF80010C1F3011101EB810100EB4100C2
:1099A00020700020E2E77CB50446022001900020F0
:1099B0000090012301AA68216B480078FEF7B4FFEC
:1099C0000546002D02DA4FF0FF307CBD01236A46C8
:1099D000682165480078FFF7AAF80546002D02DAED
:1099E0004FF0FF30F1E79DF8000000F00F009DF808
:1099F0000010C1F3011101EB810100EB4100207067
:109A00000020E2E77CB50446012001900020009090
:109A1000012301AA682154480078FEF785FF054616
:109A2000002D02DA4FF0FF307CBD01236A46682129
:109A30004D480078FFF77BF80546002D02DA4FF01D
:109A4000FF30F1E79DF8000000F00F009DF80010D6
:109A5000C1F3021101EB810100EB410020700020F5
:109A6000E2E77CB50446002001900090012301AAA2
:109A700068213D480078FEF757FF0546002D02DAC1
:109A80004FF0FF307CBD01236A46682136480078DC
:109A9000FFF74DF80546002D02DA4FF0FF30F1E7F1
:109AA0009DF8000000F00F009DF80010C1F30211B6
:109AB00001EB810100EB410020700020E2E770B56E
:109AC0000446601CFFF7CDFF0546002D02DA4FF07B
:109AD000FF3070BDA01CFFF795FF0546002D02DA90
:109AE0004FF0FF30F5E7E01CFFF75DFF0546002D66
:109AF00002DA4FF0FF30ECE7201DFFF725FF0546A7
:109B0000002D02DA4FF0FF30E3E7601DFFF7EDFEB6
:109B10000546002D02DA4FF0FF30DAE7A01DFFF70F
:109B2000B6FE0546002D02DA4FF0FF30D1E70020E7
:109B3000CFE738B5044606208DF800000A2094FBD4
:109B4000F0F100FB11400A2194FBF1F140EA011011
:109B5000C0B28DF8010002236A46682102480078ED
:109B6000FEF7E2FE054601E0B8000020002D02DA13
:109B70004FF0FF3038BD0020FCE738B50446052023
:109B80008DF800000A2094FBF0F100FB11400A213F
:109B900094FBF1F140EA0110C0B28DF801000223FC
:109BA0006A46682179480078FEF7BEFE0546002D1A
:109BB00002DA4FF0FF3038BD0020FCE738B504462C
:109BC00004208DF800000A2094FBF0F100FB114006
:109BD0000A2194FBF1F140EA0110C0B28DF80100B6
:109BE00002236A46682169480078FEF79DFE054613
:109BF000002D02DA4FF0FF3038BD0020FCE738B509
:109C0000044602208DF800000A2094FBF0F100FBCE
:109C100011400A2194FBF1F140EA0110C0B28DF825
:109C2000010002236A46682158480078FEF77CFE4E
:109C30000546002D02DA4FF0FF3038BD0020FCE76A
:109C400038B5044601208DF800000A2094FBF0F19D
:109C500000FB11400A2194FBF1F140EA0110C0B26F
:109C60008DF8010002236A46682148480078FEF713
:109C70005BFE0546002D02DA4FF0FF3038BD0020B4
:109C8000FCE738B5044600208DF800000A2094FB5C
:109C9000F0F100FB11400A2194FBF1F140EA0110C0
:109CA000C0B28DF8010002236A4668213748007867
:109CB000FEF73AFE0546002D02DA4FF0FF3038BDC0
:109CC0000020FCE770B504466078FFF7DAFF054630
:109CD000002D02DA4FF0FF3070BDA078FFF7B0FF23
:109CE0000546002D02DA4FF0FF30F5E7E078FFF788
:109CF00086FF0546002D02DA4FF0FF30ECE72079B1
:109D0000FFF75CFF0546002D02DA4FF0FF30E3E776
:109D10006079FFF732FF0546002D02DA4FF0FF3081
:109D2000DAE7A079FFF705FF0546002D02DA4FF0CC
:109D3000FF30D1E70020CFE738B508208DF80000CC
:109D400020208DF8010002236A4668210F48007820
:109D5000FEF7EAFD0446002C02DA4FF0FF3038BD72
:109D600009208DF8000005208DF8010002236A46C5
:109D7000682106480078FEF7D7FD0446002C02DA79
:109D80004FF0FF30EBE70020E9E70000B8000020CB
:109D9000F8B504460F4615461E46012C0AD1082385
:109DA000012210212E48FEF7E7FB002210212C484B
:109DB000FEF7ADFC002003466022394600902046A5
:109DC000FFF7E2F80823012231462846FEF7D4FBCC
:109DD000002231462846FEF79AFCF8BD2DE9F041F5
:109DE00005460E4617461C46DDF8188001224146FE
:109DF0002046FEF78CFC3A4631462846FFF7B0FA7B
:109E0000002241462046FEF782FCBDE8F08170B595
:109E100004460D461646324629462046FFF73DFBCE
:109E200070BD38B504460D460E4804700020034648
:109E30006022294600900B480078FFF7A5F838BD4E
:109E400070B506460D4615B94FF0FF3070BD2A4675
:109E5000314604480078FFF783FA04462046F5E7C8
:109E600000100640B900002000B585B00320002195
:109E70004FF48072304BCDE90132CDE9031005205B
:109E800003462E4A00902E48FDF75BF9032000217F
:109E90004FF480722B4BCDE90132CDE9031006203F
:109EA0000346294A00902948FDF74BF905B000BD4B
:109EB000FAF746FCFAF72DFF04464FF47A70B4FB2C
:109EC000F0F52846FEF716FAF8F7D2FCFBF75DFC32
:109ED000F9F73EF82046FEF734FBFEF731FBFFF7BB
:109EE0002DFCFFF7C1FF03E04FF47A70FDF73EFC55
:109EF000FAE788B006A916A0F8F7E5FCF8F7CCF861
:109F0000FBF734FB032000214FF48072144BCDE9A2
:109F10000132CDE9031004200346124A0090124892
:109F2000FDF70FF907AA11A10420FDF77AFAFBF754
:109F300014FC00BFFEE700004C330020483700202F
:109F4000759F00004C370020483B0020919F000087
:109F5000544D3443313239344E43504454000000A0
:109F60004C2F002048330020B19E000053746172D2
:109F70007400000008E00548FFF7A1FD002301225E
:109F800019461846FDF724FCF5E70000BA0000204A
:109F90001FB51BE00E48407800900D488378C278CA
:109FA0000CA101A800F0B6F8002405E001A8015DAD
:109FB0000C48F7F7DFFF641C01A8005D0028F5D10D
:109FC0000023012219461846FDF702FCE2E70000D3
:109FD000BA000020253032753A253032753A2530E6
:109FE0003275000000D000402DE9F05F05460020EA
:109FF00092469B4688460646814640241BE02846FA
:10A0000041464746224600F045F853465A46C01A94
:10A01000914110D311461846224600F02CF82D1A13
:10A0200067EB01084F4622460120002100F023F88B
:10A0300017EB00094E41201EA4F10104DFDC484665
:10A0400031462A464346BDE8F09F30B50B460146EF
:10A0500000202022012409E021FA02F59D4205D3C7
:10A0600003FA02F5491B04FA02F52844151EA2F171
:10A070000102F1DC30BD202A04DB203A00FA02F1B3
:10A08000002070479140C2F1200320FA03F31943E6
:10A0900090407047202A04DB203A21FA02F0002188
:10A0A000704721FA02F3D040C2F1200291400843E8
:10A0B00019467047064C074D06E0E06840F0010382
:10A0C00094E8070098471034AC42F6D3F6F79CF8B2
:10A0D0003CAE00005CAE000030B58C1810F8012BCF
:10A0E00012F00F0301D110F8013B120906D110F84C
:10A0F000012B03E010F8015B01F8015B5B1EF9D155
:10A1000001E001F8013B521EFBD1A142E6D3002041
:10A1100030BD00000FB4084B10B504A902AA039883
:10A1200000F01CF8044602A9002000F0B8F920460F
:10A1300010BC5DF814FB00009FA4000002E008C8FA
:10A14000121F08C1002AFAD170477047002001E0B1
:10A1500001C1121F002AFBD1704700002DE9FF4FFB
:10A160008BB088460546002606E025280BD0DDE9A1
:10A170000D1290476D1C761C28780028F5D10FB081
:10A180003046BDE8F08F0024A146A2460122AE4928
:10A1900000E0044315F8013F203B02FA03F00842B7
:10A1A000F7D128782A2810D06FF02F022878A0F154
:10A1B0003001092915D809EB890102EB410144F06E
:10A1C000020400EB01096D1CF0E758F8041B5FEA7C
:10A1D000010903D544F40054C9F1000944F0020414
:10A1E0006D1C28782E2817D115F8010F44F00404AF
:10A1F0002A280ED06FF02F022878A0F1300109290B
:10A200000AD80AEB8A0102EB410100EB010A6D1C3E
:10A21000F2E758F804AB6D1C28786C280FD006DCE8
:10A220004C2817D068280DD06A2814D104E074286F
:10A2300010D07A280FD10DE044F400140AE044F461
:10A24000801401E044F440146978814202D104F59D
:10A2500080146D1C6D1C2878692865D006DC0028E8
:10A260008DD0632827D0642806D15DE06E2808D001
:10A2700073282AD0752877D0DDE90D129047761C17
:10A28000E0E0C4F30250022809D003280DD0D8F82A
:10A29000001004280DD00E6008F10408D2E0D8F8B0
:10A2A0000010F217C1E90062F6E7D8F800100E803E
:10A2B000F2E70E70F0E718F8041B8DF8001000208C
:10A2C0008DF80100EB46012003E058F804BB4FF085
:10A2D000FF3061074FF0000701D40AE07F1C5745AB
:10A2E0000DDA8742FADB1BF807100029F6D106E0E9
:10A2F0007F1C8742FCDB1BF807100029F8D1DDE941
:10A300000D23A9EB07008146214600F0B1F8304447
:10A31000C61904E0DDE90D121BF8010B90477F1E02
:10A32000F8D22146484688E058F8040BC4F302519D
:10A330004FF00A0B032900D100B2042900D140B22A
:10A34000002802DA40422D2102E0210505D52B210B
:10A350008DF82410012104E006E0E10710D020214F
:10A36000F6E708AF089113E058F8040BC4F3025164
:10A370004FF00A0B032900D180B2042900D1C0B2EA
:10A380000021EEE75946FFF760FE303107F8011D66
:10A390000028F7D1ADEB070000F1200B600702D5D4
:10A3A00024F4803401E04FF0010ADA4502DDAAEB23
:10A3B0000B0000E00020824600EB0B0108980144EE
:10A3C000A9EB01000A90E00306D4DDE90D23214644
:10A3D0000A9800F04DF806444FF0000908E009A97A
:10A3E00011F80900DDE90D12904709F10109761C09
:10A3F00008998945F3DBE0030CD5DDE90D232146FF
:10A400000A9800F035F8064404E0DDE90D1230202A
:10A410009047761CBAF10001AAF1010AF5DC05E0CB
:10A42000DDE90D1217F8010B9047761CBBF1000116
:10A43000ABF1010BF4DC0A982146DDE90D2300F0B5
:10A4400005F806446D1C97E6092801002DE9F04146
:10A45000044600251E461746880404D405E0394604
:10A460002020B0476D1C641EF9D52846BDE8F08158
:10A470002DE9F041044600251E469046C80301D54B
:10A48000302700E02027880404D505E041463846FF
:10A49000B0476D1C641EF9D52846BDE8F0810A68F6
:10A4A000531C0B601070704700400040100000000B
:10A4B0000080054010000000005000401100000026
:10A4C00000900540110000000060004012000000F4
:10A4D00000A00540120000000070004013000000C2
:10A4E00000B00540130000000040024014000000CE
:10A4F00000C0054014000000005002402E00000083
:10A5000000D005402E000000006002402F00000037
:10A5100000E005402F000000007002403000000005
:10A5200000F005403000000000D00340460000006D
:10A5300000000640460000000010064047000000F2
:10A540000020064048000000003006407F00000068
:10A5500000400640800000000050064084000000DB
:10A56000006006408C000000004000401000000029
:10A570000080054010000000005000401100000065
:10A580000090054011000000006000401200000033
:10A5900000A0054012000000007000401300000001
:10A5A00000B005401300000000400240140000000D
:10A5B00000C0054014000000005002402E000000C2
:10A5C00000D005402E000000006002402F00000077
:10A5D00000E005402F000000007002403000000045
:10A5E00000F005403000000000D0034043000000B0
:10A5F0000000064043000000001006404400000038
:10A6000000200640450000000030064058000000D1
:10A610000040064059000000005006405C00000069
:10A620000060064064000000007006406C000000FE
:10A63000008006406D000000009006407F00000092
:10A640000040004000800540005000400090054060
:10A650000060004000A005400070004000B00540D0
:10A660000040024000C005400050024000D00540BC
:10A670000060024000E005400070024000F005402C
:10A6800000D00340000006400010064000100640C5
:10A690000020064000200640003006400030064002
:10A6A0000040064000400640005006400050064072
:10A6B00000600640006006400070064000700640E2
:10A6C0000080064000800640009006400090064052
:10A6D0000000024018000000001002403500000099
:10A6E00000200240540000000030024055000000ED
:10A6F00000000C407D00000000100C407E000000B7
:10A700000000024018000000001002403500000068
:10A71000002002404D000000003002404E000000CA
:10A7200000000C405600000000100C4057000000D4
:10A7300000200C407600000000300C407700000044
:10A7400000800B407D00000000900B407E00000068
:10A7500000070000000600000005000000040000E3
:10A7600000030000000200000001000000000000E3
:10A770000000000018ED00E01CED00E020ED00E01E
:10A7800000E400E004E400E008E400E00CE400E0A1
:10A7900010E400E014E400E018E400E01CE400E051
:10A7A00020E400E024E400E028E400E02CE400E001
:10A7B00030E400E034E400E038E400E03CE400E0B1
:10A7C00040E400E044E400E048E400E04CE400E061
:10A7D00050E400E054E400E058E400E05CE400E011
:10A7E00060E400E064E400E068E400E06CE400E0C1
:10A7F00070E400E074E400E078E400E07CE400E071
:10A8000080E400E084E400E088E400E000E100E0AF
:10A8100004E100E008E100E00CE100E010E100E00C
:10A8200080E100E084E100E088E100E08CE100E00C
:10A8300090E100E000E200E004E200E008E200E075
:10A840000CE200E010E200E080E200E084E200E0E0
:10A8500088E200E08CE200E090E200E040420F007D
:10A8600000201C0080841E0000802500999E360078
:10A870000040380000093D0000803E0000004B0011
:10A88000404B4C0000204E00808D5B0000C05D00FE
:10A890000080700000127A0000007D008096980011
:10A8A000001BB7000080BB00C0E8CE00647ADA006D
:10A8B0000024F4000000FA0080A81201002D3101EC
:10A8C00000366E0140787D0140000000000000006D
:10A8D000000100003E000800000000000001000030
:10A8E000A00000000200000000010000345401003C
:10A8F00000000000000100002B70060000000000B6
:10A90000000100002800000000000000000100001D
:10A9100027000100000000000001000020000000EE
:10A9200000000000000100005000000002000000D4
:10A93000000100001AAC000000000000000100004F
:10A94000179409000000000000010000169805009F
:10A9500000000000000100001400000000000000E2
:10A96000000100001380080000000000000100004A
:10A97000A00000000800000000010000100000001E
:10A98000000000000001000028000000020000009C
:10A990000001000040000000040000000001000071
:10A9A0006000000000000000000100005D000C00DD
:10A9B0000000000000010000500000000000000046
:10A9C000000100004E000200000000000001000035
:10A9D00041AC010000000000000100003C0000004C
:10A9E00000000000000100003A80090000000000A3
:10A9F0000001000030000000000000000001000025
:10AA000028000000000000000001000027000100F5
:10AA100000000000000100002360060000000000AC
:10AA2000000100002160080000000000000100009B
:10AA30001E00000000000000000100001DC0040016
:10AA400000000000000100005000000002000000B3
:10AA500000010000180000000000000000010000DC
:10AA60001400000000000000000100006000000071
:10AA700004000000000100000024F4003000300059
:10AA8000005A62029100910000879303D200D20025
:10AA900000B4C4041301130100E1F505540154018D
:10AAA000000E27079501950100688909001C4E0ECC
:10AAB00000C000401500000000D00040160000005B
:10AAC00000E000403100000000F000404B000000BA
:10AAD000000001404C000000001001404D0000004B
:10AAE000002001404E000000003001404F000000F7
:10AAF00000C000401500000000D00040160000001B
:10AB000000E000403100000000F00040480000007C
:10AB10000000014049000000001001404A00000010
:10AB2000002001404B000000003001404C000000BC
:10AB300008070606050505050404040404040404C6
:10AB400003030303030303030303030303030303D5
:10AB500002020202020202020202020202020202D5
:10AB600002020202020202020202020202020202C5
:10AB700001010101010101010101010101010101C5
:10AB800001010101010101010101010101010101B5
:10AB900001010101010101010101010101010101A5
:10ABA0000101010101010101010101010101010195
:10ABB0000000000000000000000000000000000095
:10ABC0000000000000000000000000000000000085
:10ABD0000000000000000000000000000000000075
:10ABE0000000000000000000000000000000000065
:10ABF0000000000000000000000000000000000055
:10AC00000000000000000000000000000000000044
:10AC10000000000000000000000000000000000034
:10AC20000000000000000000000000000000000024
:10AC300078563412FFFFFFFFFFFFFFFFFFFFFF7F8C
:10AC400055555555FFFFFF3F33333333AAAAAA2A80
:10AC500024499224FFFFFF1F1CC7711C9999991961
:10AC600074D1451755555515133BB113922449120C
:10AC700011111111FFFFFF0F0F0F0F0F8EE3380E91
:10AC80005E43790DCCCCCC0C0CC3300CBAE8A20BD3
:10AC90002C64210BAAAAAA0AA3703D0A899DD8098F
:10ACA0005E427B0949922409B0DCD3088888880871
:10ACB00084104208FFFFFF077CF0C10787878707E2
:10ACC00007755007C7711C07000001000200010052
:10ACD0000300010002000100040001000200010065
:10ACE0000300010002000100050001000200010054
:10ACF0000300010002000100040001000200010045
:10AD00000300010002000100060001000200010032
:10AD10000300010002000100040001000200010024
:10AD20000300010002000100050001000200010013
:10AD30000300010002000100040001000200010004
:10AD400003000100020001000700010002000100F1
:10AD500003000100020001000400010002000100E4
:10AD600003000100020001000500010002000100D3
:10AD700003000100020001000400010002000100C4
:10AD800003000100020001000600010002000100B2
:10AD900003000100020001000400010002000100A4
:10ADA0000300010002000100050001000200010093
:10ADB0000300010002000100040001000200010084
:10ADC0000300010002000100010000007856341267
:10ADD0000100400001001800000601000100100001
:10ADE000140002000A0001003F00010001000500FC
:10ADF00001001800780001000400010004001800A0
:10AE000008000100040001000100010080000100B1
:10AE10001600010001008000010001000100400057
:10AE20005800E80301001A72010010000100080038
:10AE3000E803280080020800400022195CAE0000F0
:10AE4000000000206C060000D8A000006CAE0000DE
:10AE50006C060020E43600004CA1000001FF01FF59
:0CAE600001FF01FF01FF01FF017900006C
:0400000500000201F4
:00000001FF
